:1000000002686032000000000000000265C60000C7
:10001000000000320000000000000002273F000046
:100020000000000233C100000000000266A20000D0
:1000300050523330324C434420763131302E35200B
:100040004864773A462034303030752032392D30CC
:10005000352D30342031323A34342020284329528F
:100060006F6765722053702E4A2E207777772E7235
:100070006F6765722E706C2C2074656C2F666178CA
:10008000202B34382035352032373230313332208E
:100090002843296A502D706C2C204D6F6E61204CC6
:1000A0006973612043452C2049534F393030312C3E
:1000B0002031737420436C617373D320202052204D
:1000C00045205320452054D25052333032204C43E7
:1000D0004420763131302E35002D2D2F2D2D202D21
:1000E0002D3A2D2D004350523A20004C6F633A2098
:1000F000004C4F433A2000D22020202020202020F6
:100100002020202020202020D200454E545259206B
:10011000202000455849542020202000445554599F
:10012000204558495400494E5445524E414C00D147
:1001300020202020202020202020202020202020BF
:10014000D1435243202020204520722072206F206E
:10015000720020202020200020D1466C617368208E
:10016000435243204572726F722000D3436F6E6614
:100170006967204D656D204572726F7200D3205300
:10018000657276696365204F4E00D32053657276A1
:10019000696365204F464600D2204D415354455275
:1001A000204944203D20203F2000D3536574207413
:1001B000696D652048484D4D202020D200D35365FD
:1001C00074206461746520524D4D44445720D20020
:1001D000D22020202020202020202020202020206D
:1001E00020D2D501055245473A200000D3D5021050
:1001F00044206F2077206E206C206F2061206420C7
:1002000000D120202020202020202020202020205D
:10021000202020D1D5030C50617373776F72643F37
:10022000203A2000D2D50410204163636573732007
:1002300064656E696564202000D2D5051020416395
:1002400063657373206772616E7465642000D1D535
:100250000410204163636573732064656E6965648F
:100260002020D2D50610204E6F204475616C2045A9
:100270006E747279202000D3D509104475616C200A
:10028000456E747279204D6F64652000D1D50A0ADD
:100290002020204572726F72202300202020200031
:1002A000D1D50C1020202041504220526573657436
:1002B0002020202000D2D50E104C696D6974206575
:1002C00078636565646564202000D50F0C4E4F523D
:1002D0004D414C20202020202000D1D5041020208A
:1002E0004143434553532044454E59202020D2D505
:1002F0001010204150422056696F6C6174696F6E16
:10030000202000D1D50D10202020204964656E7476
:10031000204F4B20202020D2D510102041504220C9
:1003200056696F6C6174696F6E202000D2D5111010
:10033000204E6F206F6E6520696E736964652020A2
:1003400000D1D51210202020557365722049442019
:100350003D203F202000D320202020552053204541
:100360002052D2D51610202050726F6772616D6DC9
:10037000696E6700D3202020494E5354414C4C45B0
:100380005220202020D2D51610202050726F677284
:10039000616D6D696E6720202000D22020202046EC
:1003A000205220452045202020202000D22020203F
:1003B0004520582049205320542053202000D1D5D7
:1003C000041020204143434553532044454E5920B7
:1003D0002020D2D506102020496E70757420426C02
:1003E0006F636B73202000D1D5041020204143435C
:1003F0004553532044454E59202020D2D507102084
:1004000020434C4F534544204D4F4445202020006D
:10041000D1D5041020204143434553532044454E39
:1004200059202020D2D508104F7574206F66207493
:10043000696D65207A6F6E6500D1D504102020416A
:1004400043434553532044454E59202020D2D50BD9
:1004500010204F464620636F6E646974696F6E208A
:100460002000D1D51310202053574954434820442D
:10047000454E59202020D2D508104F7574206F6644
:100480002074696D65207A6F6E6500D1D5041020E7
:10049000204143434553532044454E59202020D208
:1004A000D5141020202020505245414C41524D205F
:1004B00020202000D1D5151020537769746368651A
:1004C000722049443D203F2000C28E53890F43894A
:1004D00010758BD6758D97C28FD28E308FFDC28EE0
:1004E00022C28E53890F438910758BEB758DCBC259
:1004F0008FD28E308FFDC28E22C28E53890F4389D8
:1005000010E58AC4242BF58B758DEBC28FD28E300B
:100510008FFDC28E22F9C3137004A259801814C033
:10052000E0030303540F243DF8D0E0540704F5F032
:10053000E213D5F0FCE992E02275F0061205E922FB
:10054000C2A075F0061205E9D2A0221205401205DC
:1005500039120540120539120540120539120540BD
:1005600012053912054075F0181205E922C2A0756E
:10057000F04B1205E9D2A022755B0412338FC2A0A2
:1005800075F0C81205E9D2A022755B0512338F12EF
:10059000056D75F01E1205E912056D22755B0712D7
:1005A000338F12055722755B0612338F12055D22B9
:1005B00012054B12054B22755B0712338F755B06D4
:1005C00012338F12055D12055D12055D22D209C23C
:1005D0006E12054075F0121205E9C209C26E2212B0
:1005E000054075F0121205E9221204C9202907C03E
:1005F000F0122966D0F0D5F0F0227004A259B3228F
:10060000C0E014120609D0E022C0E0030303540F37
:1006100028F8D0E0C0E0540704F5F0E213D5F0FC70
:10062000D0E02212054B75F0641204C9D5F0FA220D
:1006300012055775F0C81204C9D5F0FA80F22230BD
:100640002316C223C2AC1204F91204F9D29912077C
:1006500009C266D2B61266AD301D16C21DC2AC12FA
:1006600004F91204F9D29912162AC266D2B6126699
:10067000AD301F16C21FC2AC1204F91204F9D29990
:100680001216AFC266D2B61266AD301E16C21EC2B8
:10069000AC1204F91204F9D29912154BC266D2B603
:1006A0001266AD302016C220C2AC1204F91204F951
:1006B000D29912158DC266D2B61266AD302116C21D
:1006C00021C2AC1204F91204F9D2991216F7C266CB
:1006D000D2B61266AD302216C222C2AC1204F91292
:1006E00004F9D29912178AC266D2B61266ADE57BBA
:1006F0006013B40105122FE38008B40205122FF233
:100700008000757B0012296622126516C2B6753804
:10071000007403124183E51E124183E51F124183D9
:100720007450124183747D124183900000E536605D
:100730000F9003E81460099007D0146003900BB881
:100740007E7D7F0875F000C0F0126511B40203D3FE
:100750008001C3D0E033F5F0A3DFEC124183DEE289
:10076000E5381241833099FD22C0F075F0DCD5F0F8
:1007700008B2041219A0125ECDC0F01209FBD0F02D
:1007800030E7EBD0F022AAF0120769E5336530F5C7
:10079000F0E534653145F0600C1208E085303385B2
:1007A00031341207691209AE1207691209E2120701
:1007B000691208F38AF022AAF0120769E53365305E
:1007C000F5F0E534653145F0600C1208E085303312
:1007D0008531341207691209941207691209E2126D
:1007E00007691208F38AF022792075300175310308
:1007F0007532E090007B1207691208E01207691257
:10080000095C790075300175310475320090009BE8
:100810001207691208E012076912095C79E0753065
:100820000175310575320090019B1207691208E0CD
:1008300012076912095C85303385313422AAF0121F
:100840000769E5336530F5F0E534653145F0600C56
:100850001208E085303385313412076912093E8A67
:10086000F022AAF0120769E5336530F5F0E534654A
:100870003145F0600C1208E08530338531341207C1
:10088000691209208AF022C0F075F00833C29792ED
:10089000A600D297D5F0F5D0F022C0F075F008C2CE
:1008A00097D29700A2A133D5F0F5D0F022D205D28D
:1008B00097D2A6D2A1D2061219A022E53133E53093
:1008C0003322C3E5313322E532221208871208BBF6
:1008D0001208871208C21208871208C71208872256
:1008E0001208ADC2061219A074531208CAD2061219
:1008F00019A0221208ADC2061219A074581208CA13
:10090000D2061219A0221208ADC2061219A0745400
:100910001208CAE412088712089AD2061219A022F5
:100920001208ADC2061219A074541208CAE41208C3
:100930008712089AF608D9F9D2061219A0221208CD
:10094000ADC2061219A074541208CAE41208871224
:10095000089AF208D9F9D2061219A0221208ADC2DB
:10096000061219A074541208CAE412088712089AD1
:10097000F0A3D9F9D2061219A0221208ADC0E0C224
:10098000061219A074841208CAD0E0120887D20691
:100990001219A0221208ADC2061219A074841208FE
:1009A000CAE612088708D9F9D2061219A02212083D
:1009B000ADC2061219A074841208CAE21208870890
:1009C000D9F9D2061219A0221208ADC2061219A036
:1009D00074841208CAE0120887A3D9F9D206121942
:1009E000A0221208ADC2061219A074831208CAD23E
:1009F000061219A01204C91204C922C2061219A0B3
:100A0000745712088712089AD2061219A022D2A689
:100A1000D2A1D297D205D2061219A0B2041219A0FF
:100A200075F0021204C9D5F0FAC205B2041219A079
:100A300075F0021204C9D5F0FAD205B2041219A059
:100A4000227530017531DB753200120769120CE234
:100A50007533FF7534FF22AE83AD8290DB007F20BB
:100A60007404F9747DF87530018583318582321202
:100A70000862787DE66E702508E66D702008E660F5
:100A80001AB4FF028013167404F9747DF8753001EE
:100A90008583318582321207B7C322D322A3A3A351
:100AA000A3DFBD80F490DB007F207404F9747DF82F
:100AB000753001858331858232120862787DE66E59
:100AC000700908E66D700408E6FC22A3A3A3A3DF67
:100AD0000A7CFF2290DB007F207BFF7404F9747D89
:100AE000F8753001858331858232120862787DE69F
:100AF0006E702C08E66D702708ECB4FF0D787D76DB
:100B0000FF0876FF0876FF0874FFF67404F9747D19
:100B1000F87530018583318582321207B7C322BB55
:100B2000FF10787DE6B4FF0A08E6B4FF05C3742021
:100B30009FFBA3A3A3A3DFA3BBFF02D322EB23232B
:100B400054FC2400F5827583DB50020583787DEE2A
:100B5000F608EDF608ECF608E4F67404F9747DF88E
:100B60007530018583318582321207B7C3227583C0
:100B70000075F08E753002858331753200C0F0C08B
:100B800083120769120CE2D0830583D0F0D5F0E41C
:100B900075830075F0DA753003858331753200C0D6
:100BA000F0C083120769120CE2D0830583D0F0D520
:100BB000F0E47533FF7534FF22758300758200758C
:100BC000F08EC0F0C082C0837530028583317532EB
:100BD000001207691208E0D083D082C082C08375FA
:100BE00030008582317532001207691209E2D08324
:100BF000D08205830582D0F0D5F0C7758300758259
:100C00000075F0DAC0F0C082C0837530038583318F
:100C10007532001207691208E0D083D082C082C00A
:100C2000837530018582317532001207691209E23D
:100C3000D083D08205830582D0F0D5F0C77533FF0D
:100C40007534FF2275830075820075F08EC0F0C088
:100C500082C08375300085833175320012076912B6
:100C600008E0D083D082C082C08375300285823193
:100C70007532001207691209E2D083D0820583051C
:100C800082D0F0D5F0C775830075820075F0DAC0A8
:100C9000F0C082C083753001858331753200120740
:100CA000691208E0D083D082C082C083753003858A
:100CB00082317532001207691209E2D083D08205B1
:100CC000830582D0F0D5F0C77533FF7534FF22124B
:100CD00008ADC2061219A074501208CAD206121921
:100CE000A0221208ADC2061219A074811208CAD23D
:100CF000061219A0221208ADC2061219A07484129D
:100D000008CAE8120887D9FAD2061219A022AAF056
:100D1000120769E5336530F5F0E534653145F0607B
:100D20000C1208E0853033853134120769120CF556
:100D30001207691209E28AF0221208ADC2061219DE
:100D4000A074541208CAE4120887E4C0E012089A9A
:100D5000D0F025F0D9F5D2061219A02275830075BE
:100D600082028006758300758200E475F08D8582AD
:100D700030858331753200C082C083C0F0C0E0127C
:100D800007691208E01207697900120D39D0F025C1
:100D9000F0D0F0D083D0820583D5F0D28582308523
:100DA0008331753200C0E01207691208E01207694A
:100DB0007920120D39D0F025F07533FF7534FF22FC
:100DC0007583007582038006758300758201E47562
:100DD000F0DA858230858331753200C082C083C0ED
:100DE000F0C0E01207691208E01207697900120DDD
:100DF00039D0F025F0D0F0D083D0820583D5F0D261
:100E00007533FF7534FF05E02275830075F00075BA
:100E10003000858331753200C0F0C083120769123B
:100E20000CE2D0830583D0F0D5F0E47533FF753440
:100E3000FF75830075F0DA753001858331753200F6
:100E4000C0F0C083120769120CE2D0830583D0F092
:100E5000D5F0E47533FF7534FF221205637556FA39
:100E60003090FA75F0051204C9D5F0FA7556FA20DB
:100E700090FA22E578B406FAC083C082C0E074D14B
:100E8000126C14D0E0D082D083C083C082C0E074E2
:100E900028126C14D0E0D082D083E58312593DE54E
:100EA0008212593DC083C082C0E07429126C14D0F4
:100EB000E0D082D0837800E212593DC083C082C066
:100EC000E0742F126C14D0E0D082D0837801E2124B
:100ED000593DC083C082C0E07420126C14D0E0D0B1
:100EE00082D083C083C082C0E0743E126C14D0E014
:100EF000D082D083C083C082C0E07420126C14D032
:100F0000E0D082D0837802E212593D120E5A22C0FC
:100F1000E0E578B4096AC083C082C0E074D3126C83
:100F200014D0E0D082D083D0E0C083C082C0E01271
:100F30006C14D0E0D082D083C083C082C0E0743A09
:100F4000126C14D0E0D082D083C083C082C0E07421
:100F500020126C14D0E0D082D083787DE612593D07
:100F600008E612593D08E612593D08E612593D08B7
:100F7000E612593D08E612593DD2AF120E5AC0E0B2
:100F8000D0E022E578B40570ED600F1414600B1406
:100F90006008146005ED2488505EC083C082C0E004
:100FA00074D3126C14D0E0D082D083E583C0821257
:100FB000593DD082E58212593DC083C082C0E074A1
:100FC0002F126C14D0E0D082D083ED12593DC08333
:100FD000C082C0E07420126C14D0E0D082D083783C
:100FE0007DE612593D08E612593D08E612593D08C2
:100FF000E612593D08120E5A2222E578B405F9EDA1
:10100000248850F4C082C083C083C082C0E074D200
:10101000126C14D0E0D082D083787DE60354012492
:1010200030C083C082C0E0126C14D0E0D082D08384
:10103000C083C082C0E0743A126C14D0E0D082D079
:1010400083E612593D08E612593DC083C082C0E0D4
:101050007420126C14D0E0D082D083C083C082C0D0
:10106000E0743E126C14D0E0D082D083D083D08262
:10107000E583C082C08312593DD083D082E582C00F
:1010800082C08312593D120E5AD083D0822222E5AB
:1010900078B40540ED2488503BC083C082C0E07422
:1010A00020126C14D0E0D082D083C083C082C0E014
:1010B000743A126C14D0E0D082D08374303079024C
:1010C0007431C083C082C0E0126C14D0E0D082D0F2
:1010D00083120E5A223014597882E6540FC0E0E68B
:1010E000C4540375F00AA4D0F025F0FD7883E630EF
:1010F000E402240A540FFE901A007F3C7404F97431
:1011000000F875300185833185823212083D780000
:10111000E26D701708E26E701208E2C42354E0F525
:10112000F07883E6541F45F0F68006A3A3A3A3DF5F
:10113000CB22126AB21210D5126AC1FEAFF012624F
:10114000197DFF0DED30E70122D27975F004A4245A
:101150007BF582E5F03400F583C082C083787DE0C2
:10116000F6A308E0F6A308E0F6A308E0F6D083D0E3
:1011700082120F83787D8683088682787DB6FF078A
:1011800008B6FF030211EBC3E58233F582E5833332
:10119000F583E58224E0F582E5833405F583787FE5
:1011A000E6704808E66044FB7402F9747DF8753017
:1011B00001858331858232120862120FF9A3A37868
:1011C0007DE60856B4FF030211EB787D86F053F0FC
:1011D0007F08E6C39EC0E0E5F09FD0F0400445F0F4
:1011E0007009787DE6A2E79279DBBD12108EBD0012
:1011F0003DB279122F714033204230202A0E304305
:101200000B205805307924800320791FA279925849
:1012100092E0A25992E1F5F013925965F030E00B9B
:101220002059051230018003123010021143ED14D1
:10123000C0E0030303540F243DF8D0E0540704FB3F
:101240007400D333DBFD307905FBE24B8004F4FB03
:10125000E25BF20211431208871208BB12088712E0
:1012600008C2D2E01208871208C7120887221208A3
:10127000ADC2061219A07454121256E41208871255
:10128000089AF608D9F9D2061219A0221208ADC29E
:10129000061219A07484121256E612088708D9F9AA
:1012A000D2061219A02290FC007530047531007529
:1012B0003200C082C0837556FA1207691208E085B1
:1012C000307A8531797908787D12076912126E12A9
:1012D00014A2D083D0827044C082C0837881868378
:1012E0000886821213534024787F868308868212F0
:1012F00013534018121372E582600AE576B5790C33
:10130000E577B57A07D083D08202132E787FE62462
:101310009AF61214E51258BFD083D0820531E53118
:1013200070020530A3E5824583708712133575334B
:10133000FF7534FF22787F7600087600788176008A
:10134000087600087600087600757A047579001230
:1013500014C122C082C083E5822400F582E5833473
:1013600080F5834005D083D08222D083D082900044
:101370000022E58275F008A4F582E5F0C58375F0DA
:1013800008A42583F583E5F03404F577E58224008D
:10139000F582E5833400F583500205778583762254
:1013A0001258CFD083D08222C082C08312147B70A7
:1013B000EF787F868308868212135340E3121372FC
:1013C0001217EF787D76007881E518F608E519F6B2
:1013D0000876000876007408F9747DF88577308502
:1013E00083318582321207B77404F97481F88577E6
:1013F0003085833185823212086275F004787D79F8
:1014000081E667600280990809D5F0F512148278A8
:101410007F8683088682A3121353787FA68308A64B
:101420008278818683088682121353787FE66583EB
:10143000700A08E665827004A31213537881A683AC
:1014400008A682C07AC07985777A8576791214C128
:10145000D0E0D0F0B57909C5F0B57A028018C5F0B2
:10146000C07AC07985F07AF579787FE62499F6120A
:1014700014E5D079D07AD083D0822212148212144B
:10148000A222857A308579317532001207691208F7
:10149000E07908787D12076912126E853033853144
:1014A00034227882E61826182618261824556670E5
:1014B0000F7882E6186618661866186618649966CA
:1014C000221214C81214E5227882E618261826186B
:1014D00026182455F67882E6186618661866186687
:1014E000186499F622857A308579317532001207B1
:1014F000691208E01207697908787D12128C1207C8
:10150000691209E21207691208F385303385313414
:101510002212147B7030787FE6C0E008E6C0E00855
:101520008683088682C3D0E09582F582D0E09583D9
:10153000F58350104582600CE5822400F582E58336
:101540003480F583C322900000D322C2B612151155
:10155000E433C0E07538007403124183E51E124184
:1015600083E51F1241837453124183D0E0124183FB
:1015700074001241837400124183E583124183E5B4
:1015800082124183E5381241833099FD22C2B6E5CB
:10159000366004F4FF8004FF1213357538007403BD
:1015A000124183E51E124183E51F124183745612D6
:1015B0004183EF124183E5381241833099FD227453
:1015C00001C0E0787D75F008E4F608D5F0FBD0E0C6
:1015D000D32212151140E860E8788186830886825C
:1015E0001215E5C322C082C083E58275F008A4F518
:1015F00082E5F0C58375F008A42583F583E5F03412
:1016000004F577E5822400F582E5833400F5835004
:101610000205777408F9747DF88577308583318504
:101620008232120862D083D082221215117F0850B4
:10163000051213357F00787F866408866508866604
:10164000088667C2B67538007403124183E51E121E
:101650004183E51F1241837454124183E5361241E0
:1016600083EF124183E536603CE5676565F5F0E59B
:1016700066656445F0600B8567828566831215E5B3
:1016800080031215C1856782856683A31213538573
:101690008267858366787D75F008E612418308D5F8
:1016A000F0F8D536C4E5381241833099FDC322E500
:1016B000367007C2AF1215115005E536F4800C786C
:1016C00081A66608A6671214C1E536D2AFC0E0C293
:1016D000B67538007403124183E51E124183E51F7D
:1016E0001241837455124183D0E0124183E53812D0
:1016F00041833099FDD322C2B6126AB275380074A4
:1017000003124183E51E124183E51F124183745782
:101710001241837882E6232354031241837883E6BF
:1017200030E402240A541F1241837882E6C4540133
:10173000F5F0A4E5F0E6540F25F01241837882E637
:10174000C45401F5F0A4E5F0E6540F25F0124183EE
:101750007880E6C45403F5F0A4E5F0E6540F25F0D4
:10176000124183787FE6C45403F5F0A4E5F0E65413
:101770000F25F01241837883E603C4540712418396
:10178000E5381241833099FDD322C2B67538007412
:1017900003124183E51E124183E51F1241837458F1
:1017A0001241837420232354FC04124183742012B9
:1017B000418390DB007F207404F9747DF87530015B
:1017C000858331858232120862787DE61241830872
:1017D000E612418308E612418308E612418308A31A
:1017E000A3A3A3DFD2E5381241833099FDD322129F
:1017F0006AB27883E630E402240A540FC4F978828E
:10180000E6C4540375F00AA4F5F0E6540F25F0C3BE
:101810001349787EF67882E692E754C0F97880E63C
:10182000C4540775F00AA4F5F0E6540F25F049F901
:101830007881E6C4540375F00AA4F5F0E6540F2548
:10184000F0F5F0787FE654702345F07880F6787FE5
:10185000E9F622C082C083C083C082C0E074D21285
:101860006C14D0E0D082D083E53012593DE53112BE
:10187000593DC083C082C0E07420126C14D0E0D007
:1018800082D083C083C082C0E07468126C14D0E040
:10189000D082D083787FE612593D08E612593DC0C8
:1018A00083C082C0E07420126C14D0E0D082D08358
:1018B000C083C082C0E07474126C14D0E0D082D0B7
:1018C0008308E612593D08E612593DC083C082C024
:1018D000E07420126C14D0E0D082D083C083C08228
:1018E000C0E07420126C14D0E0D082D083C083C0DA
:1018F00082C0E07420126C14D0E0D082D083C08308
:10190000C082C0E07420126C14D0E0D082D0831268
:101910000E5AD083D0822253630F53620F5318F0B4
:1019200053190FC2AFE5622324AEF8E5184519F646
:1019300008A61A056253620FE562B5630505635395
:10194000630FD2AF22E563B562057400780022C34D
:101950003324AEF8E6C0E008E6F8D0E02275F008DF
:101960003392A3D2A2C2A2D5F0F622E51DA2E3B320
:10197000306C029207306F02920A306E029209A216
:101980000792E0A20892E1A20A92E2A20992E3A2DF
:101990000B92E4A20D92E5A20C92E6A20292E7223B
:1019A000A2AFC2AFC0D0C0E0C0F0C2A4C2A2C2A366
:1019B000E561A20392E4A20592E5A20692E6A204E2
:1019C00092E712195DE56012195D12196B12195D2B
:1019D000D2A4C2A4D0F0D0E0D0D092AF22305A012D
:1019E000227561007560001219A020A54C7560FE7B
:1019F0007561FF7A0C1219A030A50DD3E56033F59F
:101A000060E56133F561DAEDEA602E15E060661598
:101A1000E0602B15E0605915E0605015E060471557
:101A2000E0603E15E0603515E0602C15E0602315A0
:101A3000E0601A15E06011800A74FF021A807400D9
:101A4000021A807401021A807402021A807403025E
:101A50001A807404021A807405021A807406021A2D
:101A6000807407021A807408021A807409021A80AE
:101A7000740A021A80740B021A80F544754501221B
:101A8000B544F7D545F9B4FF0280F4D25AF5468043
:101A9000EE305AFDC2A075F0061205E9D2A075F02D
:101AA000141205E9E546C25A223029037555F01291
:101AB00025D8205A07740F30290580F3121A912275
:101AC000F5F00303543FB40267E53F64086005E5A1
:101AD0003FB40D59E5F089F0C0F030141CC0E07837
:101AE00071E26013C3335005D0E0021B0C120515E0
:101AF00050F6D0E0021AF9D0E0D0F0A9F05403B4C7
:101B00000211C23CA23CB3920C021B9AD0F0A9F085
:101B1000021B9AB4010AD23CA23CB3920C021B9A5B
:101B2000B4030AB23CA23CB3920C021B9A021B986B
:101B3000B40365E54064086005E540B40DEFE5F0E9
:101B400089F0C0F030141CC0E07872E26013C33337
:101B50005005D0E0021B7612051550F6D0E0021BAE
:101B600063D0E0D0F0A9F05403B40211C23DA23D0D
:101B7000B3920D021B9AD0F0A9F0021B9AB4010A8D
:101B8000D23DA23DB3920D021B9AB40309B23DA20D
:101B90003DB3920D80048000D322C322786D75F08E
:101BA0000EE4F208D5F0FB74FF7875F27876F22235
:101BB000D24E6F20657874656E64656420202020A5
:101BC00020202020007570FF121B9CC214C213122B
:101BD0000DC8602E20142A7401F9747DF875300048
:101BE00075318C7532EE120862797DE7B4FF12C24E
:101BF0004CC24DC24EC24FC250C251C252C253C259
:101C000054221207E87401F97470F87530017531C7
:101C1000037532A0120862740EF9746DF875300104
:101C20007531037532A112083D7410F9744DF875C1
:101C300030017531037532C012083D7410F9745DBE
:101C4000F87530017531037532D012083DD214D2C7
:101C50001322797D774609774C09776E0977A0744E
:101C600004F9747DF875300075318D7532201207D6
:101C7000B77404F9747DF875300275318D753220B2
:101C80001207B722E4A22F92E0A23092E1A2319291
:101C9000E2797DF77401F9747DF875300075318C47
:101CA0007532E81207B7227401F9747DF8753000B7
:101CB00075318C7532E8120862797DE7A2E0922FC7
:101CC000A2E19230A2E2923122797DE4A23E92E03A
:101CD000A23F92E1A24092E2A22792E392E492E52F
:101CE000A24292E6A24392E7F709E4A24192E0A25F
:101CF0004492E1A24592E2A24692E3A24892E4A273
:101D00004992E5A24A92E6A24B92E7F709E4A24C77
:101D100092E0A24D92E1A24E92E2A24F92E3A25033
:101D200092E4A25192E5A25292E6A25392E7F7E41E
:101D3000A25492E0F77404F9747DF875300075319F
:101D40008C7532EC1207B7227404F9747DF8753083
:101D50000075318C7532EC120862797DE7A2E09251
:101D60003EA2E1923FA2E29240A2E39227A2E69233
:101D700042A2E7924309E7A2E09241A2E19244A283
:101D8000E29245A2E39246A2E49248A2E59249A2D9
:101D9000E6924AA2E7924B09E7A2E0924CA2E192B6
:101DA0004DA2E2924EA2E3924FA2E49250A2E5929B
:101DB00051A2E69252A2E7925309E7A2E09254227E
:101DC000797DF77401F9747DF875300075318C7583
:101DD00032E41207B7227401F9747DF8753000758A
:101DE000318C7532E4120862797DE7227401F9744E
:101DF00039F875300075318C7532FC1207B72274D2
:101E000001F97439F875300075318C7532FC12089F
:101E100062227401F9743AF875300075318D7532AB
:101E2000001207B7227401F9743AF8753000753161
:101E30008D753200120862227402F97439F8753017
:101E40000075318C7532FD12083D7402F9743BF84F
:101E500075300075318D75320112083D227402F91A
:101E60007439F875300075318C7532FD120786743F
:101E700002F9743BF875300075318D753201120727
:101E800086227401F9743BF875300075318C753217
:101E9000F01207B77401F9743CF875300075318C95
:101EA0007532F41207B77401F9743DF87530007596
:101EB000318C7532F61207B7227401F9743BF8754C
:101EC000300075318C7532F01208627401F9743C7F
:101ED000F875300075318C7532F41208627401F9AE
:101EE000743DF875300075318C7532F612086274E5
:101EF00001F9743EF875300075318C7532F21208B4
:101F000062227401F9743FF875300075318C7532B6
:101F1000F81207B77401F97440F875300075318C08
:101F20007532FA1207B77401F97441F8753000750B
:101F3000318C7532FB1207B7227401F9743FF875C2
:101F4000300075318C7532F81208627401F97440F2
:101F5000F875300075318C7532FA1208627401F927
:101F60007441F875300075318C7532FB12086222AD
:101F70007402F9741EF875300075318C7532E012F8
:101F800007B7227402F9741EF875300075318C752C
:101F900032E012086222C082C083E58275F008A494
:101FA0002420F582500205F0A8F0E58375F008A41E
:101FB000282400F583787D76FF7401F9747DF87527
:101FC00030008583318582321207B7A3A3A3A3A370
:101FD0007401F9747DF87530008583318582321281
:101FE00007B7D083D082C213220809E7C4F5F06690
:101FF000540F700D08E7F5F066540F7004DAEAE448
:1020000022E6540FC5F0540FC395F09212740122CA
:10201000788279277A03E6C4540FF309E6540FF364
:102020000908DAF2792778A17A06E6540FF6E36612
:1020300070080908DAF4E4C26022792C78A67A06DE
:10204000C3E3961918DAFA9212792C78A67A06E385
:10205000540FB40F08E6540FB40F108008E6540F65
:10206000B40F0B80061819DAE680CB740122C3E3A3
:1020700096B40902801214600FC3E3F5F0E695F000
:10208000B4090280031470E3E9B42704E4D26022A7
:102090001918E366540F60F080D1122010701A30C6
:1020A000601720411575185085831985821A1219F9
:1020B000177554B4D25CD25FE42204227408F97418
:1020C0007DF875300075318C7532C01208627895D4
:1020D000797D7A05121FEB227408F9747DF875304A
:1020E0000075318C7532C012086212209A22740574
:1020F000F9747DF875300075318C7532C01207B7F0
:10210000227403F97482F875300075318C7532C50C
:102110001207B722C082C083E5822420F582E583BE
:10212000347DF5837401F97442F87530008583318C
:10213000858232120862D083D082C082C083E58259
:1021400075F008A42420F582500205F0A8F0E5837C
:1021500075F008A4282400F5837408F9747DF875D7
:102160003000858331858232120862D083D082228A
:10217000C082C083E58275F008A42420F582500255
:1021800005F0A8F0E58375F008A4282400F5837411
:1021900008F97495F875300085833185823212080C
:1021A00062D083D08222C082C083E58275F008A409
:1021B0002420F582500205F0A8F0E58375F008A40C
:1021C000282400F5837406F9747DF8753000858342
:1021D00031858232120862D083D082227405F9746C
:1021E0007DF87530007531007532201208627895DF
:1021F000797D7A05121FEB22751B20751C0090005B
:10220000007405F9747DF8753000851C31851B322A
:102210001208627895797D7A05121FEB6018E51B2C
:102220002408F51B5002051CA3E583B40FD3E582F7
:10223000B4A0CE740122122114E42220130280B82B
:10224000751B00751C0075749F75750FE574251B53
:10225000C2E0F582E575351CF583C082C083E58256
:102260002400F582E583341BF5837402F9747DF84C
:10227000753001858331858232120862787D8683CC
:102280000886821221147895797D7A05121FEB70E9
:1022900005D0F0D0F022D083D082C3E58313F5833C
:1022A000E58213F582201214E58245836023E582DE
:1022B00024FFF574E58334FFF5758007A385821B41
:1022C00085831CC3E574951BE575951C40030222AC
:1022D0004C740122751B25751C009000007403F9D5
:1022E0007482F8753000851C31851B321208621229
:1022F000209A6018E51B2408F51B5002051CA3E575
:1023000083B40FD9E582B4A0D4740122122114E45D
:102310002278A1E6540FB40F030223AB20130280EE
:10232000B3751B00751C0075749F75750FE57425DA
:102330001BC2E0F582E575351CF583C082C083E5DC
:10234000822400F582E583343BF5837402F9747DC1
:10235000F8753001858331858232120862787D8676
:102360008308868212211412209A7005D0F0D0F0D2
:1023700022D083D082C3E58313F583E58213F582EF
:10238000201214E58245836022E58224FFF574E57E
:102390008334FFF5758007A385821B85831CC3E505
:1023A00074951BE575951C40028082740122789516
:1023B0007A0579A9E6540FC4F5F008E6540F45F004
:1023C000F70809DAEF22D207C26CD20AC26FD2092B
:1023D000C26ED2A075F0021204C9D5F0FA20A0474F
:1023E000C0E0EAC0E0C083C0829000BA126C70D036
:1023F00082D083D0E0AAE0D0E0D229C207C26CD25A
:102400000AD26FC209C26EC208C26D120563B2045D
:102410001219A075F00F1204C9D5F0FA30A0EC1211
:10242000249BC2AF026841D2A0120D64700712242F
:1024300062121BC522C2297556FA75F0641204C9CE
:10244000D5F0FAC2A0D20AC26F75F0641204C9D5E1
:10245000F0FAD2A0C20AC26FD2A01204E130A0806A
:1024600080D3121CA7121D48121DD6A2E09255A2BD
:10247000E19256A2E29257121DFF121E25121EB9BA
:10248000121F39121E38121F8322D207C26CD20AC1
:10249000C26FD209C26EC208C26D22D22912576021
:1024A00040E8D207C26CD20AC26FD209C26EC2081B
:1024B000C26DC01EC01F787D9000007A08E6F0084B
:1024C000A3DAFA1224F0787D9000007A08E0F6088A
:1024D000A3DAFA9000001250191220EE122101D056
:1024E0001FD01E121F70125093121335120A412270
:1024F000120E09751E30751F30C22FC230C231C294
:102500003EC23FC240C227C242C243C241D244C2BD
:1025100045C246C248C249C24AC24BC24CC24DC261
:102520004EC24FC250C251C252C253C254783974C3
:1025300022F2087400F2783B7406F2087400F2C2CA
:1025400055C256C257753904753A09753B01753C39
:1025500002753D04753E04753F07754000754100E6
:10256000121F70121C84121CC9C2E0A25592E0A274
:102570005692E1A25792E2121DC0121DEC121E12D9
:10258000121E82121F02121E5DC214C213121C52AE
:102590001263FC22307104C271800975F00C20B303
:1025A00005D5F0FAD322C32220522C202929122546
:1025B000945024122714E8C0E0E9C0E0EAC0E075B6
:1025C0005B0075F0031204C9D5F0FA123216D0E0A0
:1025D000FAD0E0F9D0E0F822D2698008C269122668
:1025E0004C754300C228D2717556FA7440302902E6
:1025F000740CF553C268C25AE553603B1225A820FB
:10260000683575F0031204C9D5F0FA12063F202987
:102610000320281A305AE1D27820691B75536012C2
:102620001A91B40B0D75F0081204C9D5F0FAD268EE
:10263000800512263F80C1C267D2AF7556FA225379
:102640004307F8E54324A1C8F605432278A175F0B5
:102650000874FFF608D5F0FB22306709202E03D25C
:102660002E22C26722C22E22D297122672C297123F
:10267000267222C297C2B5122672D297122672D241
:10268000B5122672C29712267275F0083392B512EF
:102690002668D5F0F722D2B775F008D297122672C5
:1026A000A2B7C29712267233D5F0F022C297C2B5F4
:1026B000122672D297122672D2B5122672C29712C1
:1026C0002672D2B512266812266812266822D29780
:1026D000D2B77473122673744B1226737450122679
:1026E000731204F9740812267312269623243F30BD
:1026F0001A022420543F4480122673746B122673EE
:102700001204E174681226731204F97460122673BD
:102710001226AC22C2ABC28ED2AFD297D2B722C29F
:10272000AFC28E53890F438910758B19758DFCC20A
:102730008FD28ED2AFC264D2BBD2AB3064FD22C086
:10274000D0A2B79263D264D0D0C2ABC28EC28F7512
:102750008B0D758DFED28EC2AF32D2698004D271DC
:10276000C269C2287556FAD22D7440302902740C01
:10277000F55312264C754300C268C267C25AC26B39
:1027800012063F202903202841B20E300E1DB20F41
:10279000300F18201907122714B21AD22D20290B36
:1027A0001225A8206826206723D22D305A2BD278F4
:1027B000206919755360122714D22D121A91B40B87
:1027C0001575F0081204C9D5F0FAD26812271475ED
:1027D00056FA1260F42212263FE55360EF1261951B
:1027E000302D05C22D1226CEC28EC2ABD2AF20B77D
:1027F00005306BFA808812063F30B706306BFA025C
:10280000277E790812271F3063DE208FDB20B7FA7E
:10281000D9F27895790B7B007A057C00C262122789
:102820001F208FC420B70520630580F52063F2A226
:10283000635002B262EC33FCDAE4D92E20E0C30329
:10284000540F6B600280A17895790A75F000E65408
:102850000FF6700205F008D9F5E5F024F850028073
:1028600087D267D219D2780227CC30620820E003E1
:102870000227E8808D03540FF6086BFB809A853998
:1028800057755800B23BE5396002D23BA23BB39288
:102890000BD271223028012278A1760A08760380B3
:1028A0000778A1760A0876010875F06484F608E5D1
:1028B000F075F00A84F608A6F0754305D228227553
:1028C00018C0751900751A0112191722755200C225
:1028D0005E7518C0751900751A0212191722D25C9C
:1028E0007554B475185075190F751AFF12191722FF
:1028F000C21612287E204E0C75181075190F751A05
:10290000FF12191722204E0C75182075190F751A11
:10291000FF1219172275186075190F751AFF121911
:10292000172275187075190F751AFF12191722C022
:10293000E0EAC0E0C083C0829002A0126C70D08236
:10294000D083D0E0AAE0D0E01263FC7518C07519FE
:1029500000751A0E12191722122ACD4008122CECFB
:102960004003122EBF22302903C38006A290302FCD
:1029700001B37836E233F2B4FF028006022AD702AE
:102980002B832032032038F7D23830141CC0E07873
:102990006DE26013C3335005D0E0022B831205159E
:1029A00050F6D0E00229A9D0E0E53B60D2B4012680
:1029B000D2171228BF303B15204C0C7558027557A2
:1029C00002305003755701853A52022B83204A0387
:1029D0001228DE022B83B40215303F032059092050
:1029E00073061228F0022B75122905022B83B403FB
:1029F00008C259122915022B83B40705D27D757CB4
:102A000003B4090C205903204B03022ABF022B8375
:102A1000B40A02743DB43212122F9B7518C0751996
:102A200002855C1A121917022B75B4330B122F8111
:102A300050031228A1022B83B43408740012289486
:102A4000022B83B435087410122894022B83B436F9
:102A5000087411122894022B83B4370874201228AA
:102A600094022B83B4381B7401F9747DF87530001F
:102A700075318C7532F1120862787DE61228940265
:102A80002B83B4391B7401F9747DF87530007531EE
:102A90008C7532F1120862787DE61228A1022B8330
:102AA000B43C0612292F022B75B43D13205908D2CD
:102AB00059122922022B75C259122915022B75753C
:102AC0001890751909F51A121917022B83E53BB4F2
:102AD0000B03A23822C32270F12032033038EBC23C
:102AE0003830141CC0E0786DE26013C3335005D059
:102AF000E0022B8312051550F6D0E0022B00D0E047
:102B0000E53B6022B40107C2171228CC8075B402DD
:102B1000028070B40307D2591229228066B40908D2
:102B2000205944304B41805BB40A02743DB43202F8
:102B30008051B43302804CB43403022B83B4350388
:102B4000022B83B43603022B83B43703022B83B4E6
:102B50003803022B83B43903022B83B43C03022BCA
:102B600083B43D03022B837518A0751909F51A1259
:102B70001917022B83101003022B831263641205B2
:102B80009CD210C232302903C38006A2913030019A
:102B9000B37837E233F2B4FF028006022CF6022D3E
:102BA000A22033032039F7D23930141CC0E0786EEC
:102BB000E26013C3335005D0E0022DA21205155078
:102BC000F6D0E0022BC8D0E0E53C60D2B40126D2BA
:102BD000171228BF303B15204C0C75580275570250
:102BE000305003755701853A52022DA2204A031234
:102BF00028DE022DA2B40215303F032059092073AC
:102C0000061228F0022D94122905022DA2B4030801
:102C1000C259122915022DA2B40705D27D757C0375
:102C2000B4090C205903204B03022CDE022DA2B460
:102C30000A02743DB43212122F9B7518C075190226
:102C4000855C1A121917022D94B4330B122F815080
:102C5000031228A1022DA2B4340874001228940291
:102C60002DA2B435087410122894022DA2B436088F
:102C70007411122894022DA2B437087420122894DB
:102C8000022DA2B4381B7401F9747DF875300075FB
:102C9000318C7532F5120862787DE6122894022D87
:102CA000A2B4391B7401F9747DF875300075318C4C
:102CB0007532F5120862787DE61228A1022DA2B4C1
:102CC0003C0612292F022D94B43D13205908D259E5
:102CD000122922022D94C259122915022D94751819
:102CE0009075190AF51A121917022DA2E53CB40BBA
:102CF00003A23922C32270F12033033039EBC239E9
:102D000030141CC0E0786EE26013C3335005D0E08D
:102D1000022DA212051550F6D0E0022D1FD0E0E5DD
:102D20003C6022B40107C2171228CC8075B402029D
:102D30008070B40307D2591229228066B409082092
:102D40005944304B41805BB40A02743DB432028076
:102D500051B43302804CB43403022DA2B4350302C3
:102D60002DA2B43603022DA2B43703022DA2B4382B
:102D700003022DA2B43903022DA2B43C03022DA2FA
:102D8000B43D03022DA27518A075190AF51A12197F
:102D900017022DA2101003022DA212636412059CCB
:102DA000D210C233302903C38006A292303101B35E
:102DB0007838E233F2B4FF028006022EC9022F5C9B
:102DC000203403203AF7D23A30141CC0E0786FE286
:102DD0006013C3335005D0E0022F5C12051550F686
:102DE000D0E0022DE7D0E0E53D60D2B40705D27D0A
:102DF000757C03B4090C205903204B03022EB10249
:102E00002F5CB40A02743DB43212122F9B7518C0A5
:102E1000751902855C1A121917022F4EB4330B1262
:102E20002F8150031228A1022F5CB43408740012C1
:102E30002894022F5CB435087410122894022F5C79
:102E4000B436087411122894022F5CB43708742029
:102E5000122894022F5CB4381B7401F9747DF87544
:102E6000300075318C7532F7120862787DE61228D1
:102E700094022F5CB4391B7401F9747DF87530002D
:102E800075318C7532F7120862787DE61228A1023E
:102E90002F5CB43C0612292F022F4EB43D1320594B
:102EA00008D259122922022F4EC259122915022F77
:102EB0004E75189075190CF51A121917022F5CE54A
:102EC0003DB40B03A23A22C32270F1203403303AFE
:102ED000EBC23A30141CC0E0786FE26013C3335089
:102EE00005D0E0022F5C12051550F6D0E0022EF25C
:102EF000D0E0E53D6009B40908205944304B4180D9
:102F00005BB40A02743DB432028051B43302804C87
:102F1000B43403022F5CB43503022F5CB4360302D1
:102F20002F5CB43703022F5CB43803022F5CB43932
:102F300003022F5CB43C03022F5CB43D03022F5C00
:102F40007518A075190CF51A121917022F5C1010BC
:102F500003022F5C12636412059CD210C2342061FC
:102F60000122C261751840751900751A00121917EF
:102F700022E53B64036008E53C64036002C322D39E
:102F8000221205DF30140C1259DA400390FFF112BF
:102F90005A1F22C05C122FB1D05C22301413125978
:102FA000DA400390FFF1125A1F5005F55C125A7671
:102FB00022E55C7005755C108023B41005755C110A
:102FC000801BB41105755C208013B42005755CFF6F
:102FD000800BB4FF05755C008003755CFF125C63B9
:102FE000E55C22C25975186075190F751AFA121925
:102FF0001722D25975187075190F751AFA12191708
:1030000022C25975186075190F751AE01219172226
:10301000D25975187075190F751AE0121917221206
:10302000310D1231A42212311A1231B122B21830EC
:10303000141CC0E07871E26013C3335005D0E00285
:10304000309012051550F6D0E002304ED0E0E53F4A
:10305000604C24F84005E53F0230A9E53FB409047F
:10306000A215803DB40A04A2178036B40C03D380A5
:1030700030B40D0B303603023127D236D38022B460
:103080000E04A216801BB40F04A27D801402312707
:10309000B40D06203603023127C236C38003A2597D
:1030A000B3923CB3920C02312730185E535A037826
:1030B0005AA2E2825C4030A2E0825D4012A2E1822C
:1030C0005E4018C23CA23CB3920C7600023127B697
:1030D0000102801D76017559408016B602028011EA
:1030E00076027559A0800AB60302800576037559E9
:1030F000CCE55923F55920E00AC23CA23CB3920C1E
:10310000023127D23CA23CB3920C023127E53FB4F6
:103110000B07D23CA23CB3920C22E53FB40B07C292
:103120003CA23CB3920C2230141CC0E07872E260E6
:1031300013C3335005D0E002318812051550F6D084
:10314000E0023146D0E0E540604C24F84005E5401F
:103150000231A1E540B40904A215803DB40A04A2DD
:10316000178036B40C03D38030B40D0B3037030214
:1031700031BED237D38022B40E04A216801BB40F06
:1031800004A27D80140231BEB40D06203703023143
:10319000BEC237C38003A259B3923DB3920D023130
:1031A000BE0231BEE540B40B07D23DA23DB3920D45
:1031B00022E540B40B07C23DA23DB3920D2222C0CE
:1031C000F075F0FAD5F0FD75F064D5F0FDD0F02281
:1031D0001231BF1231BF1231BF1231BF1231BF12D3
:1031E00031BF22756A08A2E7B39293C2B41231BF0D
:1031F000C293D2B41231BFC0E0E430B30104003056
:10320000B301040030B30104D36003D5E001C3D09F
:10321000E033D56AD122D2B4C293D2B31231BFC245
:10322000B41231D0D2B41231D0205206202903304A
:10323000782A788D7601087480F608A20792E43027
:10324000520274B3F674800830520274B0F608303B
:1032500052027480F608F608F602329D788D7603E5
:10326000087680087480A26C92E5A20792E4202977
:103270000B207808A26F92E1A23B92E0F6087480DE
:1032800020291120780EE55B54074480A26E92E558
:10329000A20992E4F6087480F608F608F675F007BD
:1032A000788D7E007F00E62EFEE61231E3F62FFFDA
:1032B00008D5F0F2EED3331231E3F8EFD333687070
:1032C00062788DB6FF5D056CE56C24FE5014756C5C
:1032D00002202B0ED22B7518C0751900751A031217
:1032E0001917205206202903307803023378789387
:1032F000E620E35720E24720E17E788EE6B60078AC
:1033000008B64274D27D757C037518B075190075C6
:103310001A001219177518C0751900751A071219B5
:10332000178055E56C6014D56C11302B0EC22B75CF
:1033300018C0751900751A04121917023378788E9F
:10334000864308D26879A17A048008788ED267799A
:10335000957A05D27775F00FE6C4540FF755F0F55E
:10336000F009E6540FF755F0F5F00908DAEAE5F050
:10337000B40F051977EEC267D2B4C29375F0051287
:1033800004E120B3061204E130B303D5F0F12220AA
:10339000520C75F0031204C9D5F0FA12321622202D
:1033A000520F30770C7518B0751900751A00121984
:1033B00017227005756F1E8002D22422C298C2990E
:1033C000322029F8309918C2992066057535008099
:1033D0000EC0E0C0D075D01012369FD0D0D0E02003
:1033E000980132C2982066FAC0D0C0E0E8C0E03050
:1033F0006505C265754900E55024FE40037550021D
:10340000E54920E712E54954072324A8C0E07400E9
:103410003435C0E0E59922543F2323249BC0E07457
:10342000003434C0E0E59922156E02359A02359ACF
:10343000D56EFAB54F08D21B7549000235A002358A
:10344000B8B462FA02359A02359AB42AF102359A72
:10345000F56E24C6E56E40E624F5E56E50E0056E97
:1034600002359A7820F2156E02359A7821F2156E9F
:1034700002359A7822F2156E02359A7823F2156E8B
:1034800002359A7824F2156E02359A7825F2156E77
:1034900002359A7826F2156E02359A0235CE000270
:1034A0003441000234470002344A00023450000222
:1034B0003428000234280002342800023428000294
:1034C00034630002346B000234730002347B000268
:1034D00034830002348B0002349300023430000243
:1034E0003430000234300002343000023430000244
:1034F0003430000234300002343000023430000234
:103500003430000234300002343000023430000223
:103510003430000234300002343000023430000213
:103520003430000234300002343000023430000203
:1035300034300002343000023430000234300002F3
:1035400034300002343000023430000234300002E3
:1035500034300002343000023430000234300002D3
:1035600034300002343000023430000234300002C3
:1035700034300002343000023430000234300002B3
:1035800034300002343000023430000234300002A3
:10359000343000023430000235CE0549254FF54F56
:1035A000D0E0F8D0E0D0D032800E802A802D80305C
:1035B000803280348040803EB40908754F007549E0
:1035C0000080D7B44208754F0075498080CC754F94
:1035D0000075490080CAB51EDF80BFB51FDA80BA0A
:1035E000F54A80B6F54B80B2B54FCD7550201235F7
:1035F000F875490080AA80D6854A371266D2D2660D
:10360000E537B44603024203B447041266E822B425
:10361000500D854B361266ADC2ACC266D22322B4C1
:103620005311854B36E54B70091266ADC2ACC266CC
:10363000D21E22B4540D854B361266ADC2ACC266A2
:10364000D21D22B4550D854B361266ADC2ACC26692
:10365000D21F22B4560D854B361266ADC2ACC2667F
:10366000D22022B4570D854B361266ADC2ACC2666D
:10367000D22122B4580D854B361266ADC2ACC2665B
:10368000D22222B44E05854B36E54B24BF24E640BA
:1036900004854B3622C26622C5382538C53822E556
:1036A0003524F0400EE5352324BEC0E074003436E6
:1036B000C0E022759906C266753500D2B622803602
:1036C000803B803D803F80408045804D804F8058CA
:1036D000805680548052804D8057800D80157535FE
:1036E00003F599123698053522A836E630002CE20B
:1036F00002371B023762753800740380E4E51E80D0
:10370000E0E51F80DC0237A7E53875350F80D2125F
:1037100019451233B2883680C8E53680C1E536A235
:103720005992E080B9753503A8360536E676FF80F4
:10373000B0E536C313602714700BA23892E0B39241
:10374000E1440480D614700BA23992E0B392E144B4
:103750000880C8147008A23A92E0440C80BD74FC42
:1037600080B9E5361470107408A27292E0A27392C8
:10377000E1A23B92E280A41470107410A23892E08F
:10378000A23992E1A23A92E280911470087418A2D0
:103790002B92E0808614700BA27492E0A27592E1E5
:1037A00002371BE402371BE537B4410675350402C6
:1037B00036E1B4422AE536600330241B53620F53CE
:1037C000630FC2AFE563B56206D2AFD30237D70548
:1037D0006353630FD2AFC3756F1E74420236DEB4FB
:1037E00044552014F7E536C3137022B39270122F9C
:1037F00071404020423D30430B20580530703480EA
:103800000320702FA270925992580238339270148C
:10381000C0E0030303540F243DF8D0E0540704FA3A
:103820007400D333DAFD307005FAE24A8004F4FA0A
:10383000E25AF6E53780A5B44B0280030238CCE5A6
:103840003654F8B40812E536540760371460431450
:10385000604714605C0236B3B4200FE5365407604D
:103860005914605C14605F0236B3B42813E536A2C5
:10387000E09259757B015003757B02E5370236DE15
:103880000236B3751AF4C273C272755701755801C6
:10389000805E751AF3D27380EF751AF2D272C2731A
:1038A000755701755801C23BA23BB3920BD2718090
:1038B0003F751AF1D272C2738031C274C2758039F9
:1038C000D274C2758033C274D275802DB4430FB5E3
:1038D00036037551037535077536A90236E1B44ACA
:1038E00020E5367019207316751AF0C21612287E5C
:1038F00075181075190F121917E5370236DE0236E2
:10390000B3B445067535060236E1B4510675350C7B
:103910000236E1B44D0EE536121AC0E5375002B258
:10392000E70237DCB44C0675350E0236E1B44602C8
:1039300080C9B4470280C4B44F08C25CC25DC25E95
:1039400080B9B45908C20075350D0236E1B45A0881
:10395000D20075350D0236E10236B3E571C27B60E7
:1039600002D27BE55CF55DC25F2067093068030227
:1039700039BD023F471205CD1223AE12223B702003
:1039800020740820751712403850121205A612250F
:10399000DC30680CE543600812209A7003023AF2AA
:1039A00075553CD5511475183075190085511A128A
:1039B0001917755103D25D7554B4023F191205CD24
:1039C000E54360F6B402061251F0023F47207756F5
:1039D000202803304450B4013A78A1E6B40A34C038
:1039E0005C122F9B123FC14012E543B4010878A13D
:1039F000E6B40A0280EBD05C023EDAD0E0E55CF58A
:103A00005D12059C7518C0751903855C1A1219178B
:103A1000023F47B4051078A1B60A0B08B601028030
:103A200008B603028003023AC508E675F00AA40846
:103A30002675F00AA40826C5F0703B78A2B60339B3
:103A4000202809C0F0123FC1D0F0502A85F05C85D3
:103A5000F05D12059C20280F7518C0751903855C50
:103A60001A121917023F477518C0751902855C1A9A
:103A7000121917023F47023EDA202809C0F0123F10
:103A8000ADD0F050F185F05C20280E7518C0751986
:103A900006855C1A121917800C7518C075190585F2
:103AA0005C1A121917125ACF12400CC20AC26FD2F6
:103AB00009D26E1205A612275EA267726850030231
:103AC0003969023F4712231170252074082075229E
:103AD000124038501D1205A612275E3067111205DC
:103AE000CD1223AE7895797D7A05121FEB60030223
:103AF00039A0755500755103C25EC25D205F02C2D8
:103B00005CC082C0831240DFD083D0825006123E58
:103B100064023F47C082C083120A57D083D08250CC
:103B200006123E64023F47E58224CEE58334FF500F
:103B300013124026400E122F715006123E0A023F09
:103B400047023CF61229585012123E0A023CAD12AE
:103B50003DEB023CAD123DCC023CAD2073F1303F59
:103B6000032059F1E5426058E5426009231205152A
:103B70004003023B7E023BC0123DAD023CAD30141F
:103B8000F73027F43051F1A277305301B350313080
:103B9000141BC0E07876E26012C3335004D0E0809A
:103BA000D712051550F7D0E0023BADD0E0C082C07F
:103BB00083126570D083D0825006123E28023CAD3D
:103BC000302749126516A2E09225A2E19226A2773B
:103BD000305301B39211B40005201122802BB4019F
:103BE0002220111A7518C0751900751A09121917B3
:103BF000204D06123E46023CAD123F8A800E1264F2
:103C0000938009B402ED2011DB1264BC30147930CA
:103C1000141CC0E07875E26013C3335005D0E00295
:103C20003C8812051550F6D0E0023C2ED0E0207BF7
:103C300016A277927A858372858273123F6D120580
:103C4000B7757102023F47757100E5836572F5F043
:103C5000E582657345F07006123E82023CAD751830
:103C6000C0751900751A0C121917307A0C7518B036
:103C7000751900751A00121917123EC075181085B3
:103C8000721985731A121917D20AC26F123F50A205
:103C9000779216D21512287E12339F123EC07518E5
:103CA0001085831985821A12191712059C12402F4C
:103CB0005003023F47122F7140F8C207C26CD2096D
:103CC000D26EC208C26D755B0012338F122114C010
:103CD00082C08312275ED083D082206706206811BD
:103CE000023F477895797D7A05121FEB6008023F05
:103CF0001912209A70F8302724E4A22592E0A22617
:103D000092E1B403051264E88013B40205126493CF
:103D1000800BB401051264BC800312646A30141C69
:103D2000C0E07873E26013C3335005D0E0023F195E
:103D300012051550F6D0E0023D3CD0E030540FE5BE
:103D40008245836009023D4E123D8E023F47B259C3
:103D500012339F30591A75187085831985821A128B
:103D60001917D207C26CC209C26EC208C26D801890
:103D700075186085831985821A121917C207C26CDB
:103D8000C209C26ED208C26D12059C023F47126082
:103D90001CC0E0EAC0E0C083C082900462126C7074
:103DA000D082D083D0E0AAE0D0E0023E9E12601C18
:103DB000C0E0EAC0E0C083C082900410126C70D0F2
:103DC00082D083D0E0AAE0D0E0023E9E12601CC008
:103DD000E0EAC0E0C083C082900439126C70D082E7
:103DE000D083D0E0AAE0D0E0023E9E12601CC0E08A
:103DF000EAC0E0C083C0829003E7126C70D082D02A
:103E000083D0E0AAE0D0E0023E9E12601CC0E0EA4F
:103E1000C0E0C083C0829003BE126C70D082D08399
:103E2000D0E0AAE0D0E0807612601CC0E0EAC0E0FA
:103E3000C083C08290032C126C70D082D083D0E0FB
:103E4000AAE0D0E0805812601CC0E0EAC0E0C08365
:103E5000C0829002DA126C70D082D083D0E0AAE0E7
:103E6000D0E0803A12601CC0E0EAC0E0C083C082AB
:103E70009002B5126C70D082D083D0E0AAE0D0E07E
:103E8000801C12601CC0E0EAC0E0C083C0829002C7
:103E90004E126C70D082D083D0E0AAE0D0E0757171
:103EA000007572FF7573FF12301F12339F75182053
:103EB00085831985821A1219171205891230262254
:103EC000207716E55C046011146570600C7518C0ED
:103ED000751901855C1A1219172212601CC0E0EADC
:103EE000C0E0C083C08290028C126C70D082D083FC
:103EF000D0E0AAE0D0E0740012593DC0E0EAC0E092
:103F0000C083C08290029B126C70D082D083D0E0BC
:103F1000AAE0D0E0120578802E12601CC0E0EAC052
:103F2000E0C083C082900224126C70D082D083D013
:103F3000E0AAE0D0E012301F120578123026757129
:103F4000007572FF7573FFC268C267E55DF55C229C
:103F500012601CC0E0EAC0E0C083C0829002391247
:103F60006C70D082D083D0E0AAE0D0E02212601C36
:103F7000C0E0EAC0E0C083C082900277126C70D0CB
:103F800082D083D0E0AAE0D0E02212601CC0E0EA38
:103F9000C0E0C083C082900303126C70D082D083D3
:103FA000D0E0AAE0D0E075F0321205E9227408F9F9
:103FB000747DF8753001753103753298120862808E
:103FC000127408F9747DF8753001753103753290FB
:103FD0001208627882E60856085604602DC0E0EAAE
:103FE000C0E0C083C082900201126C70D082D08386
:103FF000D0E0AAE0D0E01205A61225DC306809E581
:1040000043600512209A6002C322D322C0E0EAC0B6
:10401000E0C083C082900341126C70D082D083D004
:10402000E0AAE0D0E022E582249CE58334FF22E58B
:1040300082249CE58334FF22A256E58245836010EA
:10404000E582249CE58334FF5004A2558002A257E8
:1040500022E5822582F582E5833583F583E5822595
:1040600082F582E5833583F583E5822400F582E5D8
:1040700083345BF5837404F97400F875300185832B
:104080003185823212083D227882E654C0F5837869
:1040900083E630E402240A2323543C4583F58378E5
:1040A00082E6C4540375F00AA4F5F0E6540F25F037
:1040B000030303F5F053F0E085F08254034583F5E4
:1040C000837881E6C4540375F00AA4F5F0E6540F32
:1040D00025F04582F58222C39582E5F09583221270
:1040E00040517800E2B4FF0302415F126AB212400D
:1040F00088787DA68308A6827800E2F58308E2F539
:104100008208E2F5F008E21240D7502B7800E2F581
:104110008308E2F582787D86F008E61240D75041A8
:104120007802E2F58308E2F582787D86F008E612EF
:1041300040D7402D02415F7800E2F58308E2F58226
:10414000787D86F008E61240D740167802E2F583C3
:1041500008E2F582787D86F008E61240D75002C367
:1041600022D322C5382538C53822E55524E9400830
:10417000C207C26CC20AC26F3098EFC298E59912AA
:104180004163223099FDC299F59912416322D20709
:10419000C26CD20AC26FC2B6753800740512418370
:1041A000E51E124183E51F124183221204F9120415
:1041B000F91204F912418EE537124183E5381241B4
:1041C000833099FD22120DC80241CE120D64C0E069
:1041D00012418EE537124183D0E0124183E5381257
:1041E00041833099FD221204F912418EE5371241C4
:1041F00083797DE712418309DDF9E5381241833087
:1042000099FD22751A00755519D229E53F600B54A6
:10421000F87007C23CA23CB3920CE540600B54F826
:104220007007C23DA23DB3920DD2A0C28EC28CC215
:10423000ADC2ABC2ACC2AF7581CE904245C082C0A8
:104240008375D00032D2AFD28CC0E0EAC0E0C08328
:10425000C0829001EC126C70D082D083D0E0AAE0D2
:10426000D0E0C0E0EAC0E0C083C0829000C7126C1A
:1042700070D082D083D0E0AAE0D0E01266ADC2ACAC
:10428000D2991241ABB2041219A0755519D29802F5
:1042900042B7B40922F53812416AB51E2712416AA5
:1042A000B51F2112416AB4461B12416AAF38124150
:1042B0006A6F70101241ABD2B6C207C26CC20AC29A
:1042C0006F12416AB40ACBF53812416AB51EF51275
:1042D000416AB51FEF12416AF537B46D03024367B7
:1042E000B46E03024380B46F030243B7B470030299
:1042F0004404B47103024418B47303024429B4742F
:104300000302442BB4750302443FB47603024457BE
:10431000B4770302446BB4780302447FB479030298
:1043200044A0B47A030244BCB46C030244D0B46B1E
:10433000030244F2B46A0302452DB46903024549FD
:10434000B4680302458BB467030245A3B466030255
:1043500045BEB46503024682B46403024F66B4618D
:1043600003024FC10242B7AF3812416A6F70F512B3
:1043700041ABD2B675F01E1204C9D5F0FA026841FD
:1043800012416AFD1424E0402B12416A2400FC7B98
:104390000012416AFEAF3812416A6F70178EF0ED5D
:1043A000F9747DF88B308C3185F03212086212413D
:1043B000E67555190242B712416AFD1454E070F4D3
:1043C00012416A2400FC247140EA7B0212416AFE19
:1043D000EDFA787D12416AF608DAF9AF3812416ACF
:1043E0006F70D1D207C26CD20AC26F8EF0EDF97431
:1043F0007DF88B308C3185F0321207B71241B475DD
:10440000551980B0AF3812416A6F70A8120B6E1246
:1044100041AB7555190242B7AF3812416A6F700946
:104420001241CB7555190242B7808912416AFD14B9
:1044300024E0404812416A2400FC7B0102439112AF
:10444000416AFD1454E0703412416A2400FC2425B2
:10445000402A7B030243CCAF3812416A6F701D02C1
:10446000447C1241B47555190242B7AF3812416A03
:104470006F70091241C57555190242B70243B479EC
:10448000207D0712416AF309DDFCAF3812416A6FE3
:1044900070EA12595940E5126A931241B40242B7C8
:1044A000AF3812416A6F70D4126AB21204F9124125
:1044B0008EE5371241831217130242B7AF3812410B
:1044C0006A6F70661213351241AB7555190242B707
:1044D00012416AFE12416AFD12416AFCAF38124174
:1044E0006A6F7046120AD440411241AB75551902E9
:1044F00042B712416AFE12416AFDAF3812416A6F3B
:104500007028120AA51204F91204F912418EE53737
:10451000124183EE124183ED124183EC124183E597
:10452000381241833099FD0242B70243B4AF3812CA
:10453000416A6F70F51204F91204F912418EE537E1
:104540001241831217A30242B7AF3812416A6F704B
:10455000D9120D5C60027401C0E0120DC0600274DB
:1045600002D0F045F0700A120BB9121C521213352A
:10457000E4C0E012418EE537124183D0E01241835E
:10458000E5381241833099FD0242B712416AFD14A9
:1045900054E0702712416A2400FC2471401D7B0006
:1045A0000243CC12416AFD1454E0700F12416A2498
:1045B00000FC242540057B010243CC0243B4AF3804
:1045C00012416A6F70F51204F91204F912418EE576
:1045D000371241837401124183744C124183746E0B
:1045E0001241837446124183743512418374001260
:1045F0004183748D124183742012418374DA124115
:10460000837400124183740F12418374A01241839A
:1046100074801241837400124183740012418374C8
:10462000201241837400124183740012418374008C
:10463000124183740012418374001241837400128A
:10464000418374001241837400124183740012414B
:1046500083740012418374001241837400124183F9
:1046600074001241837400124183740012418374F8
:1046700000124183E5381241833099FD0242B702AE
:1046800043B412416AF58312416AF5822460E583DE
:1046900034F040EB1249D812416AFD1454E070DF47
:1046A000780012416AF208DDF9AF3812416A6F7082
:1046B000CE1241AB75F0051204C9D5F0FA1241B41F
:1046C000751A013014B93013B6124B4B124B31121C
:1046D00049E6122114789579007A0A75F00FE354AF
:1046E0000FF652F00809DAF643F0F0E5F004789599
:1046F000797D7A05121FEB600B12479A5006751AE6
:104700000402467F124B311249E612211478A17936
:104710000A7A0675F00FE3540FF652F00809DAF63C
:1047200043F0F0E5F00478A179827A03121FEB6080
:104730000B1248385006751A0602467F124B31128A
:104740004B94751A650242B7C0E07830E583F208F1
:10475000E582F2D0E022C0E07832E583F208E5821B
:10476000F2D0E022C0E07830E2F58308E2F582D0B2
:10477000E022C0E07832E2F58308E2F582D0E02260
:10478000E5822400F582E583341BF58322E582244B
:1047900000F582E583343BF583221249E6AB83AC16
:1047A00082901B00C0837900753003858331753298
:1047B000009000361207691208E012076912095CBE
:1047C0009000367A80E0A3F5F0E0A36C7005E5F088
:1047D0006B6017DAF0D0830583740024C0E583345E
:1047E000C550C174051248E7D322D083EA2AF5F0F8
:1047F000E4C395F0F582124748789579007A0A75F6
:10480000F00FE3540FF652F00809DAF643F0F0E542
:10481000F004600C122240700A74061248E7D3229A
:10482000122240E5822582F582E5833583F58312E5
:104830004780124756024D6B1249E6AB83AC82901B
:104840003B00C08379007530038583317532009059
:1048500000361207691208E012076912095C90001D
:10486000367A80E0A3F5F0E0A36C7005E5F06B60AC
:1048700017DAF0D0830583740024C0E58334A55093
:10488000C174051248E7D322D083EA2AF5F0E4C3C5
:1048900095F0F58212474878A1790A7A0675F00FEB
:1048A000E3540FF652F00809DAF643F0F0E5F004AD
:1048B000601D122321701BAB83AC821249E6EBB55D
:1048C0008306ECB58202C32274041248E7D3221295
:1048D0002321E5822582F582E5833583F58312471E
:1048E0008D124756024D6BF51A22C082C083E583B4
:1048F00012593DD083D082C082C083E58212593DD7
:10490000C083C082C0E07420126C14D0E0D082D08A
:1049100083D083D08222C082C0837F00E58224F0CE
:10492000C0E0E58334D8C0E05007D083D0820F8048
:10493000EBD0E0D0E0C083C082C0E0EF2410126C66
:1049400014D0E0D082D0837F00E5822418C0E0E557
:104950008334FCC0E05007D083D0820F80EBD0E0DE
:10496000D0E0C083C082C0E0EF2410126C14D0E00D
:10497000D082D0837F00E582249CC0E0E58334FFB1
:10498000C0E05007D083D0820F80EBD0E0D0E0C0F1
:1049900083C082C0E0EF2410126C14D0E0D082D02B
:1049A00083E58275F00A84C0F0F5F0C083C082C050
:1049B000E0E5F02410126C14D0E0D082D083D0F067
:1049C000C083C082C0E0E5F02410126C14D0E0D0A7
:1049D00082D083D083D08222C0E07834E583F2088D
:1049E000E582F2D0E022C0E07834E2F58308E2F517
:1049F00082D0E022C083C082C0E074D3126C14D095
:104A0000E0D082D083C083C082C0E0746F126C1487
:104A1000D0E0D082D083C083C082C0E0743A126CF0
:104A200014D0E0D082D0837882E612593D7883E6B4
:104A300012593D7884E612593DC083C082C0E074AB
:104A400020126C14D0E0D082D083C083C082C0E03A
:104A50007420126C14D0E0D082D083C083C082C096
:104A6000E07420126C14D0E0D082D083C083C08266
:104A7000C0E07420126C14D0E0D082D083C083C018
:104A800082C0E074D2126C14D0E0D082D083C08394
:104A9000C082C0E0746E126C14D0E0D082D083C0AB
:104AA00083C082C0E0743A126C14D0E0D082D0830C
:104AB00078A1E612593D78A2E612593D78A3E61294
:104AC000593D78A4E612593D78A5E612593D78A6DD
:104AD000E612593D120E5A22C083C082C0E074D241
:104AE000126C14D0E0D082D083C083C082C0E07446
:104AF0002E126C14D0E0D082D083C083C082C0E07C
:104B0000746B126C14D0E0D082D083C083C082C09A
:104B1000E0746F126C14D0E0D082D083C083C08266
:104B2000C0E0746E126C14D0E0D082D083120E5AA2
:104B30002274001241837400124183740012418375
:104B4000740012418374001241832275831B7582A5
:104B50001B75F040C0F0C082C08375300185833181
:104B60007532001207691208E0D083D082C082C07B
:104B7000837530038582317532001207691209E2AC
:104B8000D083D08205830582D0F0D5F0C77533FF7E
:104B90007534FF227401F97418F87530007531000E
:104BA0007532001208627401F97419F875300175D4
:104BB00031D97532FF120862AC181249E6E5822439
:104BC00020F582E583347DF583C082C0837401F9CA
:104BD0007442F8753000858331858232120862D0C4
:104BE00083D0827401F97410F875300085833185A3
:104BF00082321207867810E2F5F0E5182542C39557
:104C0000F0F5181249E6E58275F008A42420F58233
:104C1000500205F0A8F0E58375F008A4282400F5FB
:104C2000837408F9747DF87530008583318582328C
:104C3000120862787DE5187A082608DAFCF51878FB
:104C40009579007A0A75F00FE3540FF652F00809CF
:104C5000DAF643F0F0E5F00412580678A1790A7A02
:104C60000675F00FE3540FF652F00809DAF643F038
:104C7000F0E5F00412580E7408F9747DF8753000F0
:104C80008583318582321207B7787DE5187A08C3AB
:104C90009608DAFBF5181249E6C3E58233F582E59A
:104CA0008333F583C3E58233F582E58333F583E50A
:104CB000822400F582E583245BF583C082C083747F
:104CC00004F9747DF87530018583318582321208CC
:104CD00062D083D0827404F97412F8753001858330
:104CE00031858232120786787D7912E5197A042699
:104CF000F5F0E3C5F0C395F00809DAF3F51974018E
:104D0000F97418F87530007531007532001207B764
:104D10007401F97419F87530017531D97532FF12C3
:104D200007B775831B75821B75F040C0F0C082C049
:104D3000837530038583317532001207691208E0EC
:104D4000D083D082C082C0837530018582317532B4
:104D5000001207691209E2D083D08205830582D050
:104D6000F0D5F0C77533FF7534FF22124772E58224
:104D70008583F0124764C39582C0E0E5F09583D047
:104D8000F045F07002C3225003024E86124772C0F3
:104D9000E0C3E58224FEF582E58334FFF583D0E0AD
:104DA000124756E5828583F0124764B58207E5F025
:104DB000B58302C322124764AF83124772EFB583F3
:104DC00010AE82900034787DE0F6A308E0F6024D44
:104DD000E97EFE8F8305837402F9747DF8753003D4
:104DE00085833175320012086279007530038F3186
:104DF0007532009000361207691208E01207691236
:104E0000095C8F837582001247647D00E5836F70B3
:104E100002AD82ED2436F58275830050020583C30E
:104E2000EE9D20E05A03FCC082C083A3A3E0FAA356
:104E3000E0FBD083D082EAF0A3EBF0A3DCE9EE2420
:104E400036F58275830050020583787DE6F0A3086D
:104E5000E6F079007530038F31753200900036121C
:104E600007691209C81207691209E28530338531D2
:104E700034124772EFB58303024F5A0F024DBA74D2
:104E8000081248E7D322124764AF83124772EFB586
:104E90008310AE82900034787DE0F6A308E0F6023D
:104EA0004EBA7E008F8315837402F9747DF87530D5
:104EB000038583317532FE12086279007530038FE5
:104EC000317532009000361207691208E012076946
:104ED00012095C1247647DFEE5836F7002AD82EDBE
:104EE0002436F58275830050020583C3ED9E20E0D1
:104EF0006B03FCC0E0C3E58224FEF582E58334FF4A
:104F0000F583D0E0C082C083E0FAA3E0FBA3EAF01F
:104F1000A3EBF0D083D082DCDAEE2436F582758301
:104F20000050020583787DE6F0A308E6F07900756D
:104F300030038F317532009000361207691209C8AC
:104F40001207691209E2853033853134124772EF56
:104F5000B58303024F5A1F024E8BC32274091248B5
:104F6000E7D3220243B412416AF58312416AF58203
:104F7000AF3812416A6F70EBC01EC01F85831E855B
:104F8000821F121F707401F9747DF875300075313D
:104F900000753200120862787DE6C3951EC3951F26
:104FA000D01FD01E251E251FF67401F9747DF875DB
:104FB00030007531007532001207B71241AB024262
:104FC000B712416AF583AF3812416A6F70951204C7
:104FD000F91204F91204F912418EE5371241837473
:104FE00000124183E51A1241837400124183740058
:104FF00012418374001241837400124183E5381218
:1050000041833099FD0242B7905010C082C0833274
:105010007581CE75D000026841C082C083E58224CC
:1050200020F582E583347DF5837401F97442F875C7
:1050300030008583318582321207B7D083D082C099
:1050400082C083E58275F008A42420F58250020511
:10505000F0A8F0E58375F008A4282400F583740413
:10506000F9747DF87530008583318582321207B777
:10507000A3A3A3A3747D2404F5F07404F9E5F0F868
:105080007530008583318582321207B7D083D08294
:10509000C21322120D64C0E07401F9747DF87530FA
:1050A00000753100753200120862787DE6D0F0C3D9
:1050B00095F0F67401F9747DF8753000753100755E
:1050C00032001207B722120578C2AF80FE30141CDE
:1050D000C0E07873E26013C3335005D0E002517D25
:1050E00012051550F6D0E00250ECD0E0C0E0EAC066
:1050F000E0C083C0829004B4126C70D082D083D0A0
:10510000E0AAE0D0E0C207C26CD209D26EC208C2E7
:105110006D1205A612275E20670620683002517DB9
:105120001205DF12223B705512402F4050207408A8
:1051300020754C12403850471205A61225DC306805
:105140003CE543603812209A703302517FE543609A
:105150002C1205DF122311702412402F401F2074DF
:105160000820751B12403850161205A612275E3013
:10517000670B7895797D7A05121FEB6002D3223098
:105180005431E5824583602BE54260092312051501
:1051900040030251980251B3C0E0EAC0E0C083C0AE
:1051A00082900462126C70D082D083D0E0AAE0D0EA
:1051B000E080CAB259C312339F30591A75187085EE
:1051C000831985821A121917D207C26CC209C26EDE
:1051D000C208C26D801875186085831985821A12FD
:1051E0001917C207C26CC209C26ED208C26DC322AF
:1051F00078A1E6B40A1708E6B4055E122F714009DB
:105200001250CD400412059C221205782275F00A36
:10521000A4F5F008E625F0B4633FC207C26CD20AD9
:10522000D26FD209D26EC208C26DC0E0C0E0EAC03F
:10523000E0C083C082900198126C70D082D083D07D
:10524000E0AAE0D0E01205A612275E90000012212D
:105250001420670920682BD0E0120578221205DFA0
:105260007895797D7A05121FEB70EC30563A12056D
:10527000A61225DC3068E01205DF12209A70D802F1
:1052800052A81205DFE54360CE12209A70C930564D
:10529000171205A612275E3067BD1205DF789579D3
:1052A0007D7A05121FEB70AF1205A6C0E0EAC0E0E0
:1052B000C083C082900356126C70D082D083D0E03D
:1052C000AAE0D0E0D0E0B40B081256774056025462
:1052D000ECB40C081256B8404B0254ECB40D081252
:1052E00056E340400254ECB40E3D1256F2401CC04E
:1052F000E0EAC0E0C083C08290039A126C70D08252
:10530000D083D0E0AAE0D0E00254FBC0E0EAC0E0E5
:10531000C083C0829003AC126C70D082D083D0E086
:10532000AAE0D0E00254E8B40F52126AB2C0E0EA38
:10533000C0E0C083C0829001AA126C70D082D0837A
:10534000D0E0AAE0D0E0125864402EF824DC4029D6
:10535000E87881F6C083C082C0E0743A126C14D041
:10536000E0D082D083125864400FF824A0400AE8AD
:105370007880F6126A930254EC0254E8B41002806A
:1053800003025461126AB2C0E0EAC0E0C083C08286
:105390009001BD126C70D082D083D0E0AAE0D0E042
:1053A0001225D8205A061225D8305ACD121A91C08B
:1053B000E0C083C082C0E02410126C14D0E0D08220
:1053C000D083D0E0F824F640B0E8131354C07882BC
:1053D000F6C083C082C0E0742F126C14D0E0D0827B
:1053E000D08312586440926090F824ED408BE878A6
:1053F00083F6C083C082C0E0742F126C14D0E0D05A
:1054000082D08312586440566054F824CE404FE84E
:10541000788246F6C083C082C0E0742F126C14D02C
:10542000E0D082D0831225D8205A061225D8305ACF
:105430002D121A91C0E0C083C082C0E02410126C0B
:1054400014D0E0D082D083D0E0F824F94010E813E3
:10545000131354C0788346F6126A930254EC025434
:10546000E8B41115121AA9B4010C121AA9B407064E
:105470001257010254EC0254E8B41339203EF712DB
:10548000275E2068243067EE1220BC705BC0E0EA23
:10549000C0E0C083C082900374126C70D082D0834D
:1054A000D0E0AAE0D0E00250C6E543603B1220D82D
:1054B00070360250C6B46330121AA9B40A2A121AFE
:1054C000A9F57890017D700390018AC0E0EAC0E000
:1054D000126C70D0E0AAE0D0E075F0641204C9D577
:1054E000F0FA0254EC0254E8120578221250937537
:1054F00018C0751900751A0A12191712059C227521
:105500004200787D75F00876FF08D5F0FA22EFC0EA
:10551000E0C260789A79827A06EA30E004E6088090
:1055200002E6C4540FFFEA30E004E7098002E7C452
:10553000540FB40F10BF0F10EA6406600B20601EFA
:10554000D0E0FFE422BF0F06D0E0FF74012220600C
:10555000F7F5F08F486F6002D260DABD80DFE5F0CA
:10556000C395485002F4041460D6B408DB80D178A7
:1055700095797D7A057401B6FF02800FB7FF02802E
:105580000AE66770060809DAF8E422740122125567
:1055900099E58245837001D3228005D0E00255EA67
:1055A000121AA9C0E024F640F2D0E075F00AA4F582
:1055B000828005D0E00255EA121AA9C0E024F64024
:1055C000F2D0E0258275F00AA4F58285F08380058B
:1055D000D0E00255EA121AA9C0E024F640F2D0E069
:1055E0002582F58250020583C322D322C082C08364
:1055F00090000012217012556F701AE5828583F0B9
:10560000D083D082B5821FC5F0B5831AC082C08313
:10561000F58385F082A3E583B40FD8E582B4A0D3E7
:10562000D083D082C322D322C082C08390000012D4
:10563000217012550E701AE5828583F0D083D082D6
:10564000B5821FC5F0B5831AC082C083F58385F08B
:1056500082A3E583B40FD8E582B4A0D3D083D082EF
:10566000C322D32212275E3067311258061220EE71
:10567000C322900000800812558E401F1205A6120A
:10568000275E3067161205DF1221141258061255D4
:10569000EC4008754200125019C322D3221225DCB7
:1056A0003068F8E54324FD24FC40F012580E122126
:1056B00001C322900000800812558E40DE1205A61C
:1056C0001225DC3068D512211412580EE543600B08
:1056D00024FD24FC40C512562840C07542001250DB
:1056E00019C32212558E40081254FF125019C322BA
:1056F000D32212558E4008122114125750B322D3D0
:1057000022C21390002874D8F974FFF8753001850F
:105710008331858232120D0E75830175F01E75304E
:1057200000858331753200C0F0C083120769120C06
:10573000E2D0830583D0F0D5F0E4907D007420F9A9
:1057400074FFF8753001858331858232120D0E2287
:10575000787DE6080808080856B4FF02D322C32261
:10576000751E30751F30C277C27875F005C0F0C263
:1057700007C26CD20AD26FC209C26EC208C26D12D1
:1057800054FF12275ED0F0206709206806D5F0DDAF
:105790000257D7125826403F12059C7882E6B4FF84
:1057A00005C32275F005C0F012275ED0F020680610
:1057B000D5F0F30257D7E543B4021C78A1E624F6EE
:1057C000401508E624F6400F78A1E62430F51E08BF
:1057D000E62430F51FC322120578D32275470080D6
:1057E00003754701C25B12275E20680B30670A050C
:1057F00047E54724F550EFD322E5476007D25BB475
:105800000A027400C3227895797D7A05800678A112
:1058100079827A03E608540FC4F5F0E608540F4580
:10582000F0F709DAEF22206731306836E543600689
:1058300024FD24FC402C12580E1205A675F005C05C
:10584000F012275AD0F0206711205A06D5F0F00246
:105850005862121A91B40B0A80031258067542005E
:10586000C322D3221225D8205A061225D8305A4DE9
:10587000121A91C0E0C083C082C0E02410126C14E0
:10588000D0E0D082D083D0E0F824F640301225D882
:10589000205A061225D8305A24121A91C0E0C0832B
:1058A000C082C0E02410126C14D0E0D082D083D02B
:1058B000E0F5F024F64006E8C445F0C322D32212F6
:1058C00058CF75F0641204C9D5F0FA12054B227551
:1058D000F03C1205E9C2A075F03C1205E9D2A075B2
:1058E000F0141205E9C2A075F03C1205E9D2A075CA
:1058F000F0141205E9C2A075F0141205E9D2A075E2
:10590000F0141205E9C2A075F0141205E9D2A02224
:1059100075F00A84C0F0C083C082C0E02410126C0D
:1059200014D0E0D082D083D0F0C083C082C0E0E544
:10593000F02410126C14D0E0D082D08322C083C037
:1059400082C0E0C4540F2410126C14D0E0540F2411
:1059500010126C14D082D083227825E254C0707863
:10596000E275F00A84C445F0787FF67824E254C0EA
:105970007066E275F00A84C445F07880F67823E218
:1059800054E07054E275F00A84C445F07881F678EA
:1059900022E2604454E07040E275F00A84C445F0AD
:1059A000C0E07820E2030354C0D0F045F07882F6DE
:1059B0007821E2602354F0701FE275F00A84C44538
:1059C000F0C0E07826E254F8700EE2C42354E0D030
:1059D000F045F07883F6C322D32290000075F019C9
:1059E000C0F07402F9747DF87530018583318582C9
:1059F00032120862787EB6FF02800E18E55C301421
:105A000005B4FF02E570666011E5822410F582504E
:105A1000020583D0F0D5F0C8C322D0F0A3D3223042
:105A2000144DE58224FFF582E58334FFF58375F09C
:105A300019E5822480E58334FE5005900000800A39
:105A4000E5822410F58250020583C0F07402F974D7
:105A50007DF8753001858331858232120862787E47
:105A6000B6FF02800518E6B55C07D0F0D5F0C2C3DA
:105A700022D0F0A3D322C0E0EAC0E0C083C082906D
:105A800001D0126C70D082D083D0E0AAE0D0E07454
:105A900008F9747DF87530018583318582321208EA
:105AA00062787D7A08126CBBE5822408F582500288
:105AB00005837408F9747DF875300185833185821A
:105AC00032120862787D7A07126CBB22025B57C0E3
:105AD00083C082C0E074D1126C14D0E0D082D08335
:105AE000301BE9C21B12595940E2126A93C0E0EA26
:105AF000C0E0C083C0829000E5126C70D082D08379
:105B0000D0E0AAE0D0E0025B737822E2125910C024
:105B100083C082C0E0742F126C14D0E0D082D08396
:105B20007821E2125910C083C082C0E07420126C48
:105B300014D0E0D082D0837823E2125910C083C001
:105B400082C0E0743A126C14D0E0D082D083782402
:105B5000E2125910025C52C0E0EAC0E0C083C08289
:105B60009000EB126C70D082D083D0E0AAE0D0E03D
:105B7000126AB27882E6C45403C083C082C0E024B3
:105B800010126C14D0E0D082D083E6540FC083C0D2
:105B900082C0E02410126C14D0E0D082D083C08385
:105BA000C082C0E0742F126C14D0E0D082D0837811
:105BB00083E6C45401C083C082C0E02410126C1478
:105BC000D0E0D082D083E6540FC083C082C0E024EE
:105BD00010126C14D0E0D082D083C083C082C0E0A9
:105BE0007420126C14D0E0D082D0837881E6C45443
:105BF0000FC083C082C0E02410126C14D0E0D082A9
:105C0000D083E6540FC083C082C0E02410126C140D
:105C1000D0E0D082D083C083C082C0E0743A126CDE
:105C200014D0E0D082D0837880E6C4540FC083C003
:105C300082C0E02410126C14D0E0D082D083E654ED
:105C40000FC083C082C0E02410126C14D0E0D08258
:105C5000D08330140A1259DA5005125A7680031292
:105C60005C6322C0E0EAC0E0C083C0829001D01231
:105C70006C70D082D083D0E0AAE0D0E0E55CB4FFC5
:105C8000069002CA025CCCB4000690010A025CCC09
:105C9000B41006900113025CCCB4110690011C02F2
:105CA0005CCCB42006900126025CCCE55C75F06407
:105CB00084C0F0C083C082C0E02410126C14D0E015
:105CC000D082D083D0E0125910900152C0E0EAC0D7
:105CD000E0126C70D0E0AAE0D0E02220270122750B
:105CE00082051263FA604675F0021204C9D5F0FA13
:105CF000D582EFC0E0EAC0E0C083C08290028C127F
:105D00006C70D082D083D0E0AAE0D0E07401125948
:105D10003DC0E0EAC0E0C083C08290029B126C707C
:105D2000D082D083D0E0AAE0D0E01263FC74757812
:105D30003D1205FA502E207C2DD27CC0E0EAC0E056
:105D4000C083C0829002A0126C70D082D083D0E059
:105D5000AAE0D0E01263FC7518C0751900751A0D21
:105D600012191722C27C126AB2204504204647222B
:105D70007881E6543FF5F07939E365F0703509E351
:105D8000788066702E20472AD247C0E0EAC0E0C083
:105D900083C0829002A0126C70D082D083D0E0AA1F
:105DA000E0D0E01263FC7518C0751900751A0D1269
:105DB0001917223046437881E6543FF5F0793BE3EA
:105DC00065F0703509E3788066702E20472AD24747
:105DD000C0E0EAC0E0C083C0829002A0126C70D024
:105DE00082D083D0E0AAE0D0E01263FC7518C075C1
:105DF0001900751A0D12191722C24722C2AC1219C6
:105E0000456024F51888191213A853620F53630FC5
:105E1000C2AFE563B56206D2AFD3025E2505635318
:105E2000630FD2AFC380D7D2AC227E007F709000C8
:105E30000075F000E49325F0F5F0A3C3E5829EE53C
:105E4000839F40F0E5F0700122E5F0C0E0C083C020
:105E500082C0E074D2126C14D0E0D082D083E5838B
:105E600012593DE58212593DC083C082C0E0743AA8
:105E7000126C14D0E0D082D083C083C082C0E074A2
:105E800020126C14D0E0D082D083D0E012593DC0F3
:105E9000E0EAC0E0C083C082900158126C70D082EA
:105EA000D083D0E0AAE0D0E0C2ADC2ACD2291205C6
:105EB0006320A0FA75F0C81204C9D5F0FA30A0FD2D
:105EC00075F0C81204C9D5F0FA1266AD2275F064F7
:105ED0001209FB20E51830E315221204E1B2041286
:105EE00019A01204E1B2041219A0D5F0ED22C2AF3C
:105EF000B2041219A01204E1B2041219A01204E1B2
:105F0000D5F0CDC2A075F032125EDAD2A075F032B3
:105F1000125EDAC2A075F032125EDAD2A075F032EB
:105F2000125EDA75F096125EDA80D82230143C7474
:105F300000784D12060940337F087E007478783D62
:105F40001205FACE13CE05E0DFF4202A0E74007895
:105F50005D1206095005EE655E60108E5E8E5C7502
:105F600018C0751904855C1A12191722C2AF75186A
:105F70001075190FF51A121917D2AF2230140974BF
:105F800001784D1206095001227477783D1205FA06
:105F9000E492E0C0E07476783D1205FAD0E033FE7A
:105FA000202A0E7401785D1206095005EE655F60C7
:105FB000D78E5FEE20E10630E02E02600530E0175C
:105FC000A273727250C2C273C272755701755801C2
:105FD00074F8125F6C80B1D273C272755701755834
:105FE0000174F7125F6C80A020729DD272C273752B
:105FF0005701755801C23BA23BB3920BD27174F6A4
:10600000125F6C8083A23B827240F8D272C273C26C
:106010001612287E74F5125F6C025F88C082C083FE
:10602000C083C082C0E0126B29D0E0D082D083C090
:1060300083C082C0E0EEC0E0EFC0E0126EB6D0E0F8
:10604000FFD0E0FED0E0D082D083C0E0EEC0E0EF31
:10605000C0E0C083C082906E9E126ED0D082D0838A
:10606000D0E0FFD0E0FED0E0C083C082C0E0740C7E
:10607000126D33D0E0D082D083C083C082C0E07480
:1060800006126D1BD0E0D082D083126CCDD083D0AD
:106090008222C082C083EAC0E0E8C0E0900190EFB5
:1060A00075F010A42582F582E5F03583F583741030
:1060B000F97400F875300185833185823212083D0C
:1060C0007800E2B4FF030260E78EF0E27002742011
:1060D000C0F0126C14D0F008D5F0F0D3D0E0F8D0B6
:1060E000E0FAD083D08222C3D0E0F8D0E0FAD083A7
:1060F000D0822222C0E0E578B4010620680620673D
:106100006CD0E022C0E0EAC0E0C083C0829000F71B
:10611000126C70D082D083D0E0AAE0D0E078A1E504
:1061200043602DF9E6B40A14C083C082C0E0742A2B
:10613000126C14D0E0D082D08302614DC083C08243
:10614000C0E02410126C14D0E0D082D08308D9D4DF
:10615000C083C082C0E07423126C14D0E0D082D01F
:106160008375F0C81204C9D5F0FA026216126CCD1C
:106170007895790AE6C083C082C0E02410126C14BE
:10618000D0E0D082D08308D9EB75F0C81204C9D50D
:10619000F0FA026216C0E0E578B4027AC083C082E9
:1061A000C0E074D1126C14D0E0D082D083E4A23F5E
:1061B00092E0C083C082C0E02410126C14D0E0D002
:1061C00082D083E4A27392E0C083C082C0E0241036
:1061D000126C14D0E0D082D083E4A24392E0C0835A
:1061E000C082C0E02410126C14D0E0D082D083E4CE
:1061F000A25892E0C083C082C0E02410126C14D078
:10620000E0D082D083C083C082C0E07420126C14BE
:10621000D0E0D082D083D0E022C0E0E578B4022A7A
:10622000C083C082C0E074D2126C14D0E0D082D09F
:1062300083EF12593DEE12593DC083C082C0E07415
:1062400020126C14D0E0D082D083D0E022C0E0E5F0
:1062500078B4045302625EC0E0E578B40349C083B9
:10626000C082C0E074D2126C14D0E0D082D0837FA0
:1062700008788DE688F0C0F012593DD0F0A8F008FB
:10628000DFF17556FA305AFA121A91B40BF4C0E0E5
:10629000EAC0E0C083C0829000F7126C70D082D058
:1062A00083D0E0AAE0D0E0D0E022C083C082C0E08A
:1062B00074D1126C14D0E0D082D083C083C082C06D
:1062C000E07449126C14D0E0D082D083C083C082C5
:1062D000C0E07444126C14D0E0D082D083C083C07C
:1062E00082C0E0743A126C14D0E0D082D083E5838F
:1062F00012593DE58212593DC083C082C0E074202E
:10630000126C14D0E0D082D08322C2A075F0141297
:1063100004C9D5F0FAD2A075F0141204C9D5F0FA68
:1063200022C2A075F03C1204C9D5F0FAD2A075F0D3
:10633000141204C9D5F0FA2212630A12630A126316
:106340002112630A75F0641204C9D5F0FA221263AF
:106350002112630A12630A12630A75F0641204C9F7
:10636000D5F0FA22305909D207C26CC208C26D2298
:10637000C207C26CD208C26D2230144930141CC04E
:10638000E07874E26013C3335005D0E00263B112C9
:10639000051550F6D0E002639BD0E0D274202A03AA
:1063A0002076227518C0751900751A0F12191780FA
:1063B00014C274202A0330760C7518C07519007544
:1063C0001A10121917A2749276221208ADC2061280
:1063D00019A074541208CAE412088712089AF5F03A
:1063E0006448256833F568E5F02569B2E003F5698E
:1063F000D9E9D2061219A0222222E4227583DD7582
:10640000F010753003858331753200C083C0F012FF
:106410000769120CE2D0F0D0830583D5F0E4753320
:10642000FF7534FF1263F92202645BC082C083757A
:106430008205C0821263FAD082601CC2A075F00F80
:106440001204C9D5F0FAD2A075F0051204C9D5F02E
:10645000FAD582DE1263FCD083D082E5822400C0AC
:10646000E0E58334DDF8D0E0C32212642BC082C0A3
:1064700083F5828883787D76007401F9747DF875E0
:1064800030038583318582321207B7D083D08212E0
:1064900063F92212642BC082C083F5828883787DE1
:1064A00076027401F9747DF8753003858331858235
:1064B000321207B7D083D0821263F92212642B12F2
:1064C000642BC082C083F5828883787D7601740155
:1064D000F9747DF87530038583318582321207B7F0
:1064E000D083D0821263F92212642BC082C083F55C
:1064F000828883787D76037401F9747DF8753003A2
:106500008583318582321207B7D083D0821263F936
:1065100022126428800312642BC082C083F5828813
:10652000837401F9747DF875300385833185823277
:10653000120862787DE6B40102800CB40202800782
:10654000B4030280027400D083D082221208ADC24C
:10655000061219A074541208CAE412088712089A85
:10656000B402057568018002D9F3D2061219A0227F
:106570007568007583DD75F00F753003858331759F
:106580003200C083C0F01207691208E0120769796F
:106590000012654CD0F0D0830583E5687026D5F0F5
:1065A000D87530038583317532001207691208E00F
:1065B00012076979A012654C7533FF7534FFE568E1
:1065C0007002D322C322C28C758A45758C5DD28C31
:1065D000B20120010132C0D0C0E0C0F075D008D2B5
:1065E0006B202904E5566005B2041219A01219DDCA
:1065F000051DE51D20E03820E135202939206F04F4
:10660000A23B920AE51D30E20312302DE51D541F16
:106610007013E4B55728B55247B55456B56F5EB5FB
:106620007C60B55564E4B55645B5536BB5506CD038
:10663000F0D0E0D0D032E51D541F60E680F130503C
:106640000CE55824C24003D558CC75583CD557C6E4
:10665000C2152072C1C23BA23BB3920BD27180B66D
:10666000D552B6C2157554B4D25ED26180AB155600
:1066700080B7D554A7C25CC25DC25E809FD56F9FB4
:10668000809DD57C9DC27D8099D5559975510330EB
:106690002903025008808515538091D55091D26509
:1066A000808DC2B6206602D2B61266AD3275C800C1
:1066B000C2ADC2AC75CBFF75CA9875CDFF75CC98CD
:1066C000759853C298C299D2ACC2BC75C83475993A
:1066D000062275C800C2ACC2AD75980075CC2B758A
:1066E000CDEBD2AD75C8042275C800C2ACC2AD7581
:1066F0009800E58A242BF5CC540F658C24EBF5CD5E
:10670000D2AD75C804227580FF7590FF75A0FF7526
:106710008F01120A0ED229D2A0755700755800C2F7
:106720003BA23BB3920BC23CA23CB3920CC23DA233
:106730003DB3920DE4F542783D75F010F2D5F0FCD2
:10674000C272C273C274C275C238C239C23AC25A66
:10675000C25CC25DC25E755401755500C261D265EE
:10676000C266D26BC223C21DC21EC21FC220C24754
:10677000C221C222756D01C22BC22C755010E4F5E6
:1067800049F54AF54BF535F537751E00751F8075CF
:106790003F07754000E4F552F55AF559F562F56387
:1067A000F54575440F75460F751D0474377836F23C
:1067B0007837F27838F2D232D233D2347551037549
:1067C000530178A97A0576FF08DAFBC21B7820E42A
:1067D0007A07F208DAFCC21C755CFF855C5EC22495
:1067E000C214C249756F1E757100C27BC219C21AEC
:1067F000C215C216C217C277C278121B9C7556FA10
:10680000B2041219A07533FF7534FF757800D27C7D
:10681000757B00782F740AF2D210C27D757C0175E9
:106820008901758A3E758C5DC2B9D2A9D28CD2B667
:106830001266ADD2AFD2B4C293D2B3B2041219A0D1
:1068400022C2AF020000D6435243206C696E6961D8
:10685000203300D7435244206C696E6961203400B4
:10686000C2AF7556FAB2041219A01204E1B20412B2
:1068700019A01204E1B2041219A0D2A07581CE753C
:10688000D00012670612601CC0E0EAC0E0C083C0FE
:10689000829000C7126C70D082D083D0E0AAE0D082
:1068A000E0125E2A1263FC1223C67556FA1212A673
:1068B000755B0312338F1205B07518807519037557
:1068C0001A6E121917D22A30140F121132125F2CBD
:1068D000125F7C125CDB126379D2A0D2AFC229C2F4
:1068E0002A00000020A0091204E120A0030223E0F6
:1068F00030141530490312113230140C125F2C126F
:106900005F7C125CDB126379E5716003D57105125F
:106910005ACF800CC207C26CD209D26EC208C26DB7
:10692000E56F7006304803125DFCC26FC209C26E8B
:10693000126364C277C278D27112275E2068052084
:1069400067028030304022305D1F12601CC0E0EAD8
:10695000C0E0C083C08290048B126C70D082D08360
:10696000D0E0AAE0D0E002696C12395B782FE21522
:10697000E0F27008782F7414F20268D90268F90006
:1069800074A2126A14E8126A4FE9126A4F126A86F8
:106990002274A2126A14E8126A4FE7126A4F09D5EC
:1069A00082F8126A862274A2126A14E8126A4F747C
:1069B000A3126A14126A6FF709D58204126A86223A
:1069C000C296D297000000C29780E974A2126A149E
:1069D000E8126A4F1269D82274A3126A14126A6FFD
:1069E000F9126A862274A27A08C296000000C29741
:1069F000335005D2960269FAC296D297000000C2BF
:106A000097DAEDD29600D297000000309604C29734
:106A1000C322D3227A08D296D29700000000000049
:106A200000000000000000000000C296000000C24C
:106A300097335005D296026A3BC296D29700000067
:106A4000C297DAEDD29600D297000000C297227A60
:106A500008335005D296026A5BC296D297000000B6
:106A6000C297DAEDD29600D297000000C297227A40
:106A700008D296C29700000000D297C3309601B3A7
:106A800033DAF0C29722C296000000D297000000CD
:106A9000D29622787D76000876007881E6543FF61B
:106AA0007800797DC082758207126991D0821204C4
:106AB000C9227802797FC0827582051269A6D082C8
:106AC000227883E603C4540775F018A4C0E07881E7
:106AD000E6C4540375F00AA4F5F0E6540F25F0D08F
:106AE000F025F075F03CA4C0F0C0E07880E6C45416
:106AF0000775F00AA4F5F0E6540F25F0D0F025F064
:106B0000F5F0D0E03400C5F022000000000022C201
:106B1000ABC28E53890F438910758B60758DFFC290
:106B20008FD28E308FFDC28E22C202B2041219A003
:106B3000B2041219A01204E1B2041219A01204E165
:106B4000B2041219A01204E1B2041219A01204E155
:106B50007438F580D2A7126B09C2A7B2041219A02B
:106B60001204E17438F580D2A7126B09C2A7B204EF
:106B70001219A01204E17438F580D2A7126B09C271
:106B8000A7126B0F126B0F7438F580D2A7126B0926
:106B9000C2A7126B0F7408F580D2A7126B09C2A7A7
:106BA000126B0F7401F580D2A7126B09C2A7126B8A
:106BB0000F7406F580D2A7126B09C2A7B20412198E
:106BC000A01204E122C202B2041219A04480F5808E
:106BD000D2A7126B09C2A7126B0F22C202B2041213
:106BE00019A0547F4440F580D2A7126B09C2A712A6
:106BF0006B0F22D202B2041219A0126B0F126B0F8C
:106C0000F580D2A7126B09C2A7126B0FC202B204A1
:106C10001219A022B4D1087400126BC5026C6FB4B3
:106C2000D2087440126BC5026C6FB4D6087480121F
:106C30006BC5026C6FB4D70874C0126BC5026C6F61
:106C4000B4D306126CCD026C6FB4D41C75F00A205C
:106C50005A1DC0F075F00F1204E11204E1D5F0F7EF
:106C6000D0F0D5F0EA026C6F906D6693126BF32250
:106C7000EEC0E0EFC0E07A00EA0A936037B4D526B0
:106C8000EA603193602E14FFEA05E06027936024E8
:106C9000FE30140E12609250090A0AEA2E4015FACC
:106CA000800F0A0A800BC083C082126C14D082D07D
:106CB00083EA70C5D0E0FFD0E0FE22E6600EC0831C
:106CC000C082126C14D082D08308DAEF22C202B2E2
:106CD000041219A0C083C082C0E07401F580D2A75D
:106CE000126B09C2A7B2041219A01204E1D0E0D0BD
:106CF00082D08322C202B2041219A0C083C082C013
:106D0000E07402F580D2A7126B09C2A7B20412196F
:106D1000A01204E1D0E0D082D08322C202B20412D9
:106D200019A054034404F580D2A7126B09C2A7121C
:106D30006B0F22C202B2041219A054074408F58056
:106D4000D2A7126B09126B09C2A7126B0F22C202E3
:106D5000B2041219A0540C4410F580D2A7126B098A
:106D6000C2A7126B0F2200010203040506070809DF
:106D70000A0B0C0D0E0F30313233343536373839BB
:106D80004142434445462021222324252627282901
:106D90002A2B2C2D2E2F30313233343536373839DB
:106DA0003A3B3C3D3E3F40414243444546474849CB
:106DB0004A4B4C4D4E4F50515253545556575859BB
:106DC0005A5B5C5D5E5F60616263646566676869AB
:106DD0006A6B6C6D6E6F707172737475767778799B
:106DE0007A7B7C7D7E7FF869706C6C6C086C6C6C57
:106DF0006C6C6C096C6C6C0A0B6C6C6C6C6C6C6CF9
:106E00006C6C0D6C0D6C6C6C0C6C0F6C0F0E6C6CF8
:106E10006C6C6C6C6C6C6C6C0C0B0F6C0F0E6C08EF
:106E20006C6C6C6C6C0E6C6C0C6C0F6C0F0E6C6C78
:106E30006C6C6C6C6C6C6C6C0C6C0F6C0F0E6C6C0A
:106E40006C6C6C6C6C6C6C6C0C6C0F6C090E6C6C00
:106E50000A6C6C6C6C6C6C0F0C0C0F6C0F0E6C6C09
:106E60006C6C6C6C6C6C000E010F110F0200020454
:106E70000E1010110E00000E111F100E02000C0457
:106E800005060C040E0002040E1111110E0002047E
:106E90000E100E011E0004001F0204081F00010254
:106EA00016191111110002041F0204081F000E110F
:106EB0000102040004007406126D1B7400126BDBE7
:106EC0007E407F00906E66EF0F93126BF3DEF5222B
:106ED000C083C0827406126D1B7438126BDB7E088F
:106EE0007F00D082D083C083C082EF0F93126BF3F8
:106EF000DEF0D082D08322000000000000000000FD
:106F00000000000000000000000000000000000081
:106F10000000000000000000000000000000000071
:106F20000000000000000000000000000000000061
:106F30000000000000000000000000000000000051
:106F40000000000000000000000000000000000041
:106F50000000000000000000000000000000000031
:106F60000000000000000000000000000000000021
:106F70000000000000000000000000000000000011
:106F80000000000000000000000000000000000001
:106F900000000000000000000000000000000000F1
:106FA00000000000000000000000000000000000E1
:106FB00000000000000000000000000000000000D1
:106FC000000000000000000000000000000050521F
:106FD0003330324C434420763131302E35204864F2
:106FE000773A462034303030752032392D30352D07
:106FF00030342031323A343420204352433D007043
:00000001FF
:0300000306028072
